BL51 BANKED LINKER/LOCATER V6.22                                                        12/09/2013  13:21:20  PAGE 1


BL51 BANKED LINKER/LOCATER V6.22, INVOKED BY:
C:\KEIL4\C51\BIN\BL51.EXE ..\OBJ\main.obj, ..\OBJ\LCD drive.obj, ..\OBJ\Touch.obj TO ..\OBJ\11 PRINT (.\11.m51) RAMSIZE 
>> (256)


MEMORY MODEL: COMPACT WITH FLOATING POINT ARITHMETIC


INPUT MODULES INCLUDED:
  ..\OBJ\main.obj (MAIN)
  ..\OBJ\LCD drive.obj (LCD_DRIVE)
  ..\OBJ\Touch.obj (TOUCH)
  C:\KEIL4\C51\LIB\C51FPC.LIB (?C?FPADD)
  C:\KEIL4\C51\LIB\C51FPC.LIB (?C?FPMUL)
  C:\KEIL4\C51\LIB\C51FPC.LIB (?C?FPDIV)
  C:\KEIL4\C51\LIB\C51FPC.LIB (?C?FPCMP)
  C:\KEIL4\C51\LIB\C51FPC.LIB (?C?FCAST)
  C:\KEIL4\C51\LIB\C51FPC.LIB (?C?CASTF)
  C:\KEIL4\C51\LIB\C51FPC.LIB (SQRT)
  C:\KEIL4\C51\LIB\C51FPC.LIB (?C?FPGETOPN)
  C:\KEIL4\C51\LIB\C51C.LIB (?C_STARTUP)
  C:\KEIL4\C51\LIB\C51C.LIB (?C?CLDPTR)
  C:\KEIL4\C51\LIB\C51C.LIB (?C?UIDIV)
  C:\KEIL4\C51\LIB\C51C.LIB (?C?ISTPTR)
  C:\KEIL4\C51\LIB\C51C.LIB (?C?LMUL)
  C:\KEIL4\C51\LIB\C51C.LIB (?C?ULDIV)
  C:\KEIL4\C51\LIB\C51C.LIB (?C?LNEG)
  C:\KEIL4\C51\LIB\C51C.LIB (?C?LLDPDATA)
  C:\KEIL4\C51\LIB\C51C.LIB (?C?LSTPDATA)
  C:\KEIL4\C51\LIB\C51C.LIB (?C?LSTKPDATA)
  C:\KEIL4\C51\LIB\C51C.LIB (?C?ICALL)
  C:\KEIL4\C51\LIB\C51C.LIB (ABS)
  C:\KEIL4\C51\LIB\C51C.LIB (?C_INIT)


LINK MAP OF MODULE:  ..\OBJ\11 (MAIN)


            TYPE    BASE      LENGTH    RELOCATION   SEGMENT NAME
            -----------------------------------------------------

            * * * * * * *   D A T A   M E M O R Y   * * * * * * *
            REG     0000H     0008H     ABSOLUTE     "REG BANK 0"
            IDATA   0008H     0001H     UNIT         ?STACK

            * * * * * * *  X D A T A   M E M O R Y  * * * * * * *
            XDATA   0000H     0006H     INPAGE       ?PD?MAIN
            XDATA   0006H     0026H     INPAGE       ?PD?TOUCH
            XDATA   002CH     004BH     INPAGE       _PDATA_GROUP_

            * * * * * * *   C O D E   M E M O R Y   * * * * * * *
            CODE    0000H     0003H     ABSOLUTE     
            CODE    0003H     2890H     UNIT         ?PR?LCD_INIT?LCD_DRIVE
            CODE    2893H     090FH     UNIT         ?PR?TP_ADJUST?TOUCH
            CODE    31A2H     06C3H     UNIT         ?CO?LCD_DRIVE
            CODE    3865H     05B9H     UNIT         ?C?LIB_CODE
            CODE    3E1EH     03A1H     UNIT         ?PR?DISPLAY_ID?LCD_DRIVE
            CODE    41BFH     029DH     UNIT         ?PR?_TP_ADJ_INFO_SHOW?TOUCH
BL51 BANKED LINKER/LOCATER V6.22                                                      12/09/2013  13:21:20  PAGE 2


            CODE    445CH     0208H     UNIT         ?PR?_LCD_SETPOS?TOUCH
            CODE    4664H     01D2H     UNIT         ?PR?_LLCD_TEST_SINGLECOLOR?LCD_DRIVE
            CODE    4836H     01CFH     UNIT         ?PR?_LCD_TEST_SINGLECOLOR?LCD_DRIVE
            CODE    4A05H     01AEH     UNIT         ?PR?_LCD_DRAWLINE?TOUCH
            CODE    4BB3H     018EH     UNIT         ?PR?_LCD_SETWINDOW?LCD_DRIVE
            CODE    4D41H     018EH     UNIT         ?PR?_DRAW_CIRCLE?TOUCH
            CODE    4ECFH     0163H     UNIT         ?PR?MAIN?MAIN
            CODE    5032H     012FH     UNIT         ?PR?_TP_READ_XY2?TOUCH
            CODE    5161H     0126H     UNIT         ?PR?_TP_READ_XOY?TOUCH
            CODE    5287H     00ECH     UNIT         ?PR?_GUI_SPRINTF_CHAR?LCD_DRIVE
            CODE    5373H     00EAH     UNIT         ?PR?_TP_SCAN?TOUCH
            CODE    545DH     00E4H     UNIT         ?PR?_TP_DROW_TOUCH_POINT?TOUCH
            CODE    5541H     00DFH     UNIT         ?PR?_LCD_ID_61581?LCD_DRIVE
            CODE    5620H     00D3H     UNIT         ?PR?_LCD_SHOWNUM?TOUCH
            CODE    56F3H     00CFH     UNIT         ?CO?TOUCH
            CODE    57C2H     00CCH     UNIT         ?PR?_LCD_ID?LCD_DRIVE
            CODE    588EH     00CCH     UNIT         ?PR?_LCD_SHOWSTRING?TOUCH
            CODE    595AH     00A8H     UNIT         ?PR?SQRT?SQRT
            CODE    5A02H     00A7H     UNIT         ?PR?_LCD_ID_9341?LCD_DRIVE
            CODE    5AA9H     008CH     UNIT         ?C_C51STARTUP
            CODE    5B35H     0079H     UNIT         ?PR?_GUI_SPRINTF_STRING?LCD_DRIVE
            CODE    5BAEH     0076H     UNIT         ?PR?_LLCD_WRITE_DATA?LCD_DRIVE
            CODE    5C24H     0064H     UNIT         ?PR?_TP_READ_AD?TOUCH
            CODE    5C88H     0063H     UNIT         ?PR?_TP_DRAW_BIG_POINT?TOUCH
            CODE    5CEBH     005CH     UNIT         ?PR?_LCD_WRITE_CMD?LCD_DRIVE
            CODE    5D47H     0057H     UNIT         ?PR?_LCD_WRITE_DATA?LCD_DRIVE
            CODE    5D9EH     0053H     UNIT         ?PR?_LLCD_WRITE_CMD?LCD_DRIVE
            CODE    5DF1H     0051H     UNIT         ?PR?_DELAYMS?LCD_DRIVE
            CODE    5E42H     0049H     UNIT         ?PR?_LCD_POW?TOUCH
            CODE    5E8BH     0047H     UNIT         ?PR?_TP_READ_XY?TOUCH
            CODE    5ED2H     0046H     UNIT         ?PR?_SENG_CMD_DAT?LCD_DRIVE
            CODE    5F18H     003FH     UNIT         ?PR?_UART_SEND_DATA?LCD_DRIVE
            CODE    5F57H     003EH     UNIT         ?PR?_LCD_DRAWPOINT?TOUCH
            CODE    5F95H     003BH     UNIT         ?PR?LOAD_DROW_DIALOG?TOUCH
            CODE    5FD0H     0033H     UNIT         ?C_INITSEG
            CODE    6003H     002AH     UNIT         ?PR?LCD_READ_8347ID?LCD_DRIVE
            CODE    602DH     0029H     UNIT         ?PR?LCD_READ_ID?LCD_DRIVE
            CODE    6056H     0027H     UNIT         ?PR?LCD_READ_ID9341?LCD_DRIVE
            CODE    607DH     0020H     UNIT         ?PR?LCD_READ_ID61581?LCD_DRIVE
            CODE    609DH     001BH     UNIT         ?PR?HD_RESET?LCD_DRIVE
            CODE    60B8H     001AH     UNIT         ?PR?_TP_WRITE_BYTE?TOUCH
            CODE    60D2H     0014H     UNIT         ?PR?_GUI_POINT?LCD_DRIVE
            CODE    60E6H     0014H     UNIT         ?PR?_LCD_SETXY?LCD_DRIVE
            CODE    60FAH     000FH     UNIT         ?PR?UART_INIT?LCD_DRIVE
            CODE    6109H     000DH     UNIT         ?PR?KEYPRESS?LCD_DRIVE
            CODE    6116H     000CH     UNIT         ?PR?_DELAYUS?LCD_DRIVE
            CODE    6122H     000CH     UNIT         ?PR?_ABS?ABS



OVERLAY MAP OF MODULE:   ..\OBJ\11 (MAIN)


SEGMENT                                        PDATA_GROUP
  +--> CALLED SEGMENT                        START    LENGTH
------------------------------------------------------------
?C_C51STARTUP                                -----    -----
BL51 BANKED LINKER/LOCATER V6.22                                                      12/09/2013  13:21:20  PAGE 3


  +--> ?PR?MAIN?MAIN
  +--> ?C_INITSEG

?PR?MAIN?MAIN                                -----    -----
  +--> ?PR?LCD_READ_ID9341?LCD_DRIVE
  +--> ?PR?LCD_READ_ID61581?LCD_DRIVE
  +--> ?PR?LCD_READ_ID?LCD_DRIVE
  +--> ?PR?LCD_READ_8347ID?LCD_DRIVE
  +--> ?PR?LCD_INIT?LCD_DRIVE
  +--> ?PR?KEYPRESS?LCD_DRIVE
  +--> ?PR?DISPLAY_ID?LCD_DRIVE
  +--> ?PR?_LCD_TEST_SINGLECOLOR?LCD_DRIVE
  +--> ?PR?_TP_READ_XY?TOUCH
  +--> ?PR?_LLCD_TEST_SINGLECOLOR?LCD_DRIVE
  +--> ?PR?TP_ADJUST?TOUCH
  +--> ?PR?LOAD_DROW_DIALOG?TOUCH
  +--> ?PR?_TP_DRAW_BIG_POINT?TOUCH
  +--> ?PR?_DELAYMS?LCD_DRIVE

?PR?LCD_READ_ID9341?LCD_DRIVE                -----    -----
  +--> ?PR?HD_RESET?LCD_DRIVE
  +--> ?PR?_DELAYMS?LCD_DRIVE
  +--> ?PR?_LCD_ID_9341?LCD_DRIVE
  +--> ?PR?_UART_SEND_DATA?LCD_DRIVE

?PR?HD_RESET?LCD_DRIVE                       -----    -----
  +--> ?PR?UART_INIT?LCD_DRIVE
  +--> ?PR?_DELAYMS?LCD_DRIVE

?PR?_DELAYMS?LCD_DRIVE                       0055H    0002H
  +--> ?PR?_UART_SEND_DATA?LCD_DRIVE
  +--> ?PR?_DELAYUS?LCD_DRIVE

?PR?_UART_SEND_DATA?LCD_DRIVE                -----    -----
  +--> ?PR?UART_INIT?LCD_DRIVE

?PR?_LCD_ID_9341?LCD_DRIVE                   002CH    0006H
  +--> ?PR?_LLCD_WRITE_CMD?LCD_DRIVE
  +--> ?PR?_DELAYMS?LCD_DRIVE
  +--> ?PR?_UART_SEND_DATA?LCD_DRIVE

?PR?_LLCD_WRITE_CMD?LCD_DRIVE                -----    -----
  +--> ?PR?_LCD_WRITE_DATA?LCD_DRIVE

?PR?_LCD_WRITE_DATA?LCD_DRIVE                -----    -----
  +--> ?PR?_LCD_WRITE_CMD?LCD_DRIVE

?PR?LCD_READ_ID61581?LCD_DRIVE               -----    -----
  +--> ?PR?HD_RESET?LCD_DRIVE
  +--> ?PR?_DELAYMS?LCD_DRIVE
  +--> ?PR?_LCD_ID_61581?LCD_DRIVE
  +--> ?PR?_UART_SEND_DATA?LCD_DRIVE

?PR?_LCD_ID_61581?LCD_DRIVE                  002CH    0004H
  +--> ?PR?_LLCD_WRITE_CMD?LCD_DRIVE
  +--> ?PR?_LLCD_WRITE_DATA?LCD_DRIVE
  +--> ?PR?_DELAYMS?LCD_DRIVE
BL51 BANKED LINKER/LOCATER V6.22                                                      12/09/2013  13:21:20  PAGE 4


  +--> ?PR?_UART_SEND_DATA?LCD_DRIVE

?PR?_LLCD_WRITE_DATA?LCD_DRIVE               -----    -----
  +--> ?PR?_LLCD_WRITE_CMD?LCD_DRIVE

?PR?LCD_READ_ID?LCD_DRIVE                    -----    -----
  +--> ?PR?HD_RESET?LCD_DRIVE
  +--> ?PR?_DELAYMS?LCD_DRIVE
  +--> ?PR?_SENG_CMD_DAT?LCD_DRIVE
  +--> ?PR?_LCD_ID?LCD_DRIVE
  +--> ?PR?_UART_SEND_DATA?LCD_DRIVE

?PR?_SENG_CMD_DAT?LCD_DRIVE                  -----    -----
  +--> ?PR?_LLCD_WRITE_CMD?LCD_DRIVE
  +--> ?PR?_LLCD_WRITE_DATA?LCD_DRIVE

?PR?_LCD_ID?LCD_DRIVE                        002CH    0008H
  +--> ?PR?_LLCD_WRITE_CMD?LCD_DRIVE
  +--> ?PR?_DELAYMS?LCD_DRIVE

?PR?LCD_READ_8347ID?LCD_DRIVE                -----    -----
  +--> ?PR?HD_RESET?LCD_DRIVE
  +--> ?PR?_DELAYMS?LCD_DRIVE
  +--> ?PR?_SENG_CMD_DAT?LCD_DRIVE
  +--> ?PR?_LCD_ID?LCD_DRIVE
  +--> ?PR?_UART_SEND_DATA?LCD_DRIVE

?PR?LCD_INIT?LCD_DRIVE                       -----    -----
  +--> ?PR?_DELAYMS?LCD_DRIVE
  +--> ?PR?_SENG_CMD_DAT?LCD_DRIVE
  +--> ?PR?_LLCD_WRITE_CMD?LCD_DRIVE
  +--> ?PR?_LLCD_WRITE_DATA?LCD_DRIVE
  +--> ?PR?_LCD_TEST_SINGLECOLOR?LCD_DRIVE

?PR?_LCD_TEST_SINGLECOLOR?LCD_DRIVE          002CH    0005H
  +--> ?PR?_LCD_WRITE_DATA?LCD_DRIVE
  +--> ?PR?_LCD_WRITE_CMD?LCD_DRIVE
  +--> ?PR?_LLCD_WRITE_CMD?LCD_DRIVE
  +--> ?PR?_SENG_CMD_DAT?LCD_DRIVE
  +--> ?PR?_LLCD_WRITE_DATA?LCD_DRIVE

?PR?KEYPRESS?LCD_DRIVE                       -----    -----
  +--> ?PR?_DELAYMS?LCD_DRIVE

?PR?DISPLAY_ID?LCD_DRIVE                     -----    -----
  +--> ?CO?LCD_DRIVE
  +--> ?PR?_GUI_SPRINTF_STRING?LCD_DRIVE

?PR?_GUI_SPRINTF_STRING?LCD_DRIVE            002CH    0009H
  +--> ?CO?LCD_DRIVE
  +--> ?PR?_GUI_SPRINTF_CHAR?LCD_DRIVE

?PR?_GUI_SPRINTF_CHAR?LCD_DRIVE              0035H    000BH
  +--> ?CO?LCD_DRIVE
  +--> ?PR?_GUI_POINT?LCD_DRIVE

?PR?_GUI_POINT?LCD_DRIVE                     0040H    0002H
BL51 BANKED LINKER/LOCATER V6.22                                                      12/09/2013  13:21:20  PAGE 5


  +--> ?PR?_LCD_SETXY?LCD_DRIVE
  +--> ?PR?_LLCD_WRITE_DATA?LCD_DRIVE

?PR?_LCD_SETXY?LCD_DRIVE                     -----    -----
  +--> ?PR?_LCD_SETWINDOW?LCD_DRIVE

?PR?_LCD_SETWINDOW?LCD_DRIVE                 0042H    0006H
  +--> ?PR?_SENG_CMD_DAT?LCD_DRIVE
  +--> ?PR?_LLCD_WRITE_CMD?LCD_DRIVE
  +--> ?PR?_LLCD_WRITE_DATA?LCD_DRIVE

?PR?_TP_READ_XY?TOUCH                        003AH    0008H
  +--> ?PR?_TP_READ_XOY?TOUCH

?PR?_TP_READ_XOY?TOUCH                       0042H    0011H
  +--> ?PR?_TP_READ_AD?TOUCH

?PR?_TP_READ_AD?TOUCH                        0053H    0002H
  +--> ?PR?_TP_WRITE_BYTE?TOUCH
  +--> ?PR?_DELAYMS?LCD_DRIVE

?PR?_LLCD_TEST_SINGLECOLOR?LCD_DRIVE         004FH    0006H
  +--> ?PR?_LCD_WRITE_DATA?LCD_DRIVE
  +--> ?PR?_LCD_WRITE_CMD?LCD_DRIVE
  +--> ?PR?_LLCD_WRITE_CMD?LCD_DRIVE
  +--> ?PR?_SENG_CMD_DAT?LCD_DRIVE
  +--> ?PR?_LLCD_WRITE_DATA?LCD_DRIVE

?PR?TP_ADJUST?TOUCH                          002CH    0023H
  +--> ?PR?_LLCD_TEST_SINGLECOLOR?LCD_DRIVE
  +--> ?PR?_TP_DROW_TOUCH_POINT?TOUCH
  +--> ?PR?_ABS?ABS
  +--> ?PR?SQRT?SQRT
  +--> ?PR?_TP_ADJ_INFO_SHOW?TOUCH
  +--> ?CO?TOUCH
  +--> ?PR?_LCD_SHOWSTRING?TOUCH
  +--> ?PR?_DELAYMS?LCD_DRIVE

?PR?_TP_DROW_TOUCH_POINT?TOUCH               004FH    0004H
  +--> ?PR?_LCD_DRAWLINE?TOUCH
  +--> ?PR?_LCD_DRAWPOINT?TOUCH
  +--> ?PR?_DRAW_CIRCLE?TOUCH

?PR?_LCD_DRAWLINE?TOUCH                      0053H    001CH
  +--> ?PR?_LCD_DRAWPOINT?TOUCH

?PR?_LCD_DRAWPOINT?TOUCH                     -----    -----
  +--> ?PR?_LCD_SETPOS?TOUCH
  +--> ?PR?_LLCD_WRITE_DATA?LCD_DRIVE

?PR?_LCD_SETPOS?TOUCH                        006FH    0008H
  +--> ?PR?_SENG_CMD_DAT?LCD_DRIVE
  +--> ?PR?_LLCD_WRITE_CMD?LCD_DRIVE
  +--> ?PR?_LLCD_WRITE_DATA?LCD_DRIVE

?PR?_DRAW_CIRCLE?TOUCH                       0053H    000AH
  +--> ?PR?_LCD_DRAWPOINT?TOUCH
BL51 BANKED LINKER/LOCATER V6.22                                                      12/09/2013  13:21:20  PAGE 6



?PR?SQRT?SQRT                                004FH    0004H

?PR?_TP_ADJ_INFO_SHOW?TOUCH                  004FH    0012H
  +--> ?CO?TOUCH
  +--> ?PR?_LCD_SHOWSTRING?TOUCH
  +--> ?PR?_LCD_SHOWNUM?TOUCH

?PR?_LCD_SHOWSTRING?TOUCH                    0061H    000DH

?PR?_LCD_SHOWNUM?TOUCH                       0061H    000DH
  +--> ?PR?_LCD_POW?TOUCH

?PR?_LCD_POW?TOUCH                           006EH    0006H

?PR?LOAD_DROW_DIALOG?TOUCH                   -----    -----
  +--> ?PR?_LLCD_TEST_SINGLECOLOR?LCD_DRIVE
  +--> ?CO?TOUCH
  +--> ?PR?_LCD_SHOWSTRING?TOUCH

?PR?_TP_DRAW_BIG_POINT?TOUCH                 002CH    0004H
  +--> ?PR?_LCD_DRAWPOINT?TOUCH

?C_INITSEG                                   -----    -----
  +--> ?PR?_TP_SCAN?TOUCH
  +--> ?PR?TP_ADJUST?TOUCH
  +--> ?CO?TOUCH

?PR?_TP_SCAN?TOUCH                           -----    -----
  +--> ?PR?_TP_READ_XY2?TOUCH

?PR?_TP_READ_XY2?TOUCH                       002CH    000EH
  +--> ?PR?_TP_READ_XY?TOUCH



UNRESOLVED EXTERNAL SYMBOLS:
   ?_LCD_SHOWCHAR?BYTE
   _LCD_SHOWCHAR



SYMBOL TABLE OF MODULE:  ..\OBJ\11 (MAIN)

  VALUE           TYPE          NAME
  ----------------------------------

  -------         MODULE        MAIN
  C:0000H         SYMBOL        _ICE_DUMMY_
  D:0090H         PUBLIC        P1
  D:00B0H         PUBLIC        P3
  X:0000H         PUBLIC        tempid
  D:00A8H         PUBLIC        IE
  D:00B8H         PUBLIC        IP
  C:4ECFH         PUBLIC        main
  X:0002H         PUBLIC        zhiyi
  D:0098H         PUBLIC        SCON
BL51 BANKED LINKER/LOCATER V6.22                                                      12/09/2013  13:21:20  PAGE 7


  D:0088H         PUBLIC        TCON
  X:0004H         PUBLIC        temp
  D:00C8H         PUBLIC        T2CON
  D:00D0H         PUBLIC        PSW
  -------         PROC          MAIN
  -------         DO            
  D:0007H         SYMBOL        bawei
  D:0007H         SYMBOL        i
  -------         ENDDO         
  C:4ECFH         LINE#         10
  C:4ECFH         LINE#         11
  C:4ECFH         LINE#         14
  C:4ED5H         LINE#         17
  C:4ED8H         LINE#         18
  C:4EE1H         LINE#         19
  C:4EE1H         LINE#         20
  C:4EE4H         LINE#         21
  C:4EE4H         LINE#         24
  C:4EFEH         LINE#         25
  C:4EFEH         LINE#         26
  C:4F01H         LINE#         27
  C:4F01H         LINE#         30
  C:4F0AH         LINE#         31
  C:4F0AH         LINE#         32
  C:4F0DH         LINE#         33
  C:4F18H         LINE#         34
  C:4F18H         LINE#         35
  C:4F1FH         LINE#         36
  C:4F1FH         LINE#         37
  C:4F1FH         LINE#         38
  C:4F24H         LINE#         40
  C:4F27H         LINE#         41
  C:4F27H         LINE#         42
  C:4F2DH         LINE#         43
  C:4F30H         LINE#         44
  C:4F30H         LINE#         49
  C:4F33H         LINE#         52
  C:4F43H         LINE#         53
  C:4F43H         LINE#         55
  C:4F4DH         LINE#         56
  C:4F4DH         LINE#         57
  C:4F50H         LINE#         58
  C:4F50H         LINE#         66
  C:4F50H         LINE#         68
  C:4F5CH         LINE#         69
  C:4F5CH         LINE#         71
  C:4F66H         LINE#         72
  C:4F66H         LINE#         73
  C:4F69H         LINE#         74
  C:4F69H         LINE#         79
  C:4F71H         LINE#         80
  C:4F74H         LINE#         81
  C:4F74H         LINE#         83
  C:4F77H         LINE#         86
  C:4F7DH         LINE#         88
  C:4F8AH         LINE#         89
  C:4F8AH         LINE#         90
BL51 BANKED LINKER/LOCATER V6.22                                                      12/09/2013  13:21:20  PAGE 8


  C:4F8DH         LINE#         91
  C:4F8DH         LINE#         100
  C:4F94H         LINE#         102
  C:4FA1H         LINE#         103
  C:4FA1H         LINE#         104
  C:4FA4H         LINE#         105
  C:4FA4H         LINE#         110
  C:4FBAH         LINE#         111
  C:4FBCH         LINE#         112
  C:4FBEH         LINE#         113
  C:4FBEH         LINE#         114
  C:4FBFH         LINE#         115
  C:4FC6H         LINE#         116
  C:4FC9H         LINE#         117
  C:4FCBH         LINE#         119
  C:4FCBH         LINE#         120
  C:4FCBH         LINE#         121
  C:4FCBH         LINE#         122
  C:4FCBH         LINE#         124
  C:4FDBH         LINE#         125
  C:4FE1H         LINE#         126
  C:4FE1H         LINE#         127
  C:4FFEH         LINE#         128
  C:4FFEH         LINE#         129
  C:5013H         LINE#         130
  C:5027H         LINE#         131
  C:5027H         LINE#         132
  C:5030H         LINE#         134
  -------         ENDPROC       MAIN
  -------         ENDMOD        MAIN

  -------         MODULE        LCD_DRIVE
  C:0000H         SYMBOL        _ICE_DUMMY_
  D:0080H         PUBLIC        P0
  C:602DH         PUBLIC        LCD_read_id
  D:0090H         PUBLIC        P1
  D:00A0H         PUBLIC        P2
  D:00B0H         PUBLIC        P3
  C:607DH         PUBLIC        LCD_read_id61581
  C:5BEAH         PUBLIC        _LLCD_WRITE_DATA
  C:4664H         PUBLIC        _LLCD_TEST_SingleColor
  D:00A8H         PUBLIC        IE
  C:60A6H         PUBLIC        HD_reset
  D:00B8H         PUBLIC        IP
  B:0098H.1       PUBLIC        TI
  C:4BB3H         PUBLIC        _LCD_setwindow
  B:0090H.1       PUBLIC        RS
  C:5541H         PUBLIC        _LCD_ID_61581
  D:0099H         PUBLIC        SBUF
  D:0098H         PUBLIC        SCON
  D:0089H         PUBLIC        TMOD
  D:0088H         PUBLIC        TCON
  C:5D6CH         PUBLIC        _LCD_WRITE_DATA
  C:4836H         PUBLIC        _LCD_TEST_SingleColor
  C:57C2H         PUBLIC        _LCD_ID
  C:5DB7H         PUBLIC        _LLCD_WRITE_CMD
  C:5F4FH         PUBLIC        _UART_send_data
BL51 BANKED LINKER/LOCATER V6.22                                                      12/09/2013  13:21:20  PAGE 9


  C:3E1EH         PUBLIC        Display_ID
  C:5B4AH         PUBLIC        _GUI_sprintf_string
  D:008DH         PUBLIC        TH1
  D:008BH         PUBLIC        TL1
  C:3275H         PUBLIC        font16x8
  C:5287H         PUBLIC        _GUI_sprintf_char
  C:60D2H         PUBLIC        _GUI_Point
  C:6056H         PUBLIC        LCD_read_id9341
  C:60FAH         PUBLIC        UART_init
  B:0088H.6       PUBLIC        TR1
  C:6003H         PUBLIC        LCD_read_8347id
  B:0090H.3       PUBLIC        RDB
  C:6109H         PUBLIC        Keypress
  C:5F0AH         PUBLIC        _seng_cmd_dat
  B:0090H.0       PUBLIC        TFT_CS
  D:00C8H         PUBLIC        T2CON
  B:00B0H.3       PUBLIC        KEY
  C:0003H         PUBLIC        LCD_init
  B:0090H.4       PUBLIC        RES
  B:0090H.2       PUBLIC        WRB
  C:5E1DH         PUBLIC        _delayms
  C:5A02H         PUBLIC        _LCD_ID_9341
  C:60E6H         PUBLIC        _LCD_setxy
  C:5D15H         PUBLIC        _LCD_WRITE_CMD
  D:00D0H         PUBLIC        PSW
  C:6116H         PUBLIC        _delayus
  -------         PROC          UART_INIT
  C:60FAH         LINE#         8
  C:60FAH         LINE#         9
  C:60FAH         LINE#         10
  C:60FDH         LINE#         11
  C:6100H         LINE#         12
  C:6103H         LINE#         13
  C:6106H         LINE#         14
  C:6108H         LINE#         16
  -------         ENDPROC       UART_INIT
  C:5F22H         SYMBOL        L?0458
  -------         PROC          L?0457
  -------         ENDPROC       L?0457
  C:5F22H         SYMBOL        L?0458
  -------         PROC          _UART_SEND_DATA
  D:0007H         SYMBOL        lcdid
  C:5F4FH         LINE#         21
  C:5F4FH         LINE#         22
  C:5F4FH         LINE#         24
  C:5F51H         LINE#         25
  C:5F54H         LINE#         26
  C:5F56H         LINE#         28
  -------         ENDPROC       _UART_SEND_DATA
  -------         PROC          DISPLAY_ID
  C:3E1EH         LINE#         34
  C:3E1EH         LINE#         35
  C:3E1EH         LINE#         36
  C:3E2BH         LINE#         37
  C:3E2BH         LINE#         38
  C:3E32H         LINE#         39
  C:3E3DH         LINE#         40
BL51 BANKED LINKER/LOCATER V6.22                                                      12/09/2013  13:21:20  PAGE 10


  C:3E3DH         LINE#         41
  C:3E41H         LINE#         42
  C:3E44H         LINE#         43
  C:3E44H         LINE#         44
  C:3E48H         LINE#         45
  C:3E48H         LINE#         46
  C:3E58H         LINE#         47
  C:3E58H         LINE#         48
  C:3E5FH         LINE#         49
  C:3E6AH         LINE#         50
  C:3E6AH         LINE#         51
  C:3E6EH         LINE#         52
  C:3E70H         LINE#         53
  C:3E70H         LINE#         54
  C:3E74H         LINE#         55
  C:3E74H         LINE#         56
  C:3E77H         LINE#         57
  C:3E84H         LINE#         58
  C:3E84H         LINE#         59
  C:3E87H         LINE#         60
  C:3E92H         LINE#         61
  C:3E92H         LINE#         62
  C:3E96H         LINE#         63
  C:3E98H         LINE#         64
  C:3E98H         LINE#         65
  C:3E9CH         LINE#         66
  C:3E9CH         LINE#         67
  C:3E9FH         LINE#         68
  C:3EACH         LINE#         69
  C:3EACH         LINE#         70
  C:3EAFH         LINE#         71
  C:3EBAH         LINE#         72
  C:3EBAH         LINE#         73
  C:3EBEH         LINE#         74
  C:3EC0H         LINE#         75
  C:3EC0H         LINE#         76
  C:3EC4H         LINE#         77
  C:3EC4H         LINE#         78
  C:3ED4H         LINE#         79
  C:3ED4H         LINE#         80
  C:3EDBH         LINE#         81
  C:3EE6H         LINE#         82
  C:3EE6H         LINE#         83
  C:3EEAH         LINE#         84
  C:3EECH         LINE#         85
  C:3EECH         LINE#         86
  C:3EF0H         LINE#         87
  C:3EF0H         LINE#         88
  C:3EF3H         LINE#         89
  C:3F00H         LINE#         90
  C:3F00H         LINE#         91
  C:3F07H         LINE#         92
  C:3F12H         LINE#         93
  C:3F12H         LINE#         94
  C:3F16H         LINE#         95
  C:3F18H         LINE#         96
  C:3F18H         LINE#         97
BL51 BANKED LINKER/LOCATER V6.22                                                      12/09/2013  13:21:20  PAGE 11


  C:3F1CH         LINE#         98
  C:3F1CH         LINE#         99
  C:3F2CH         LINE#         100
  C:3F2CH         LINE#         101
  C:3F33H         LINE#         102
  C:3F3EH         LINE#         103
  C:3F3EH         LINE#         104
  C:3F42H         LINE#         105
  C:3F44H         LINE#         106
  C:3F44H         LINE#         107
  C:3F48H         LINE#         108
  C:3F48H         LINE#         109
  C:3F4BH         LINE#         110
  C:3F58H         LINE#         111
  C:3F58H         LINE#         112
  C:3F5FH         LINE#         113
  C:3F6AH         LINE#         114
  C:3F6AH         LINE#         115
  C:3F6EH         LINE#         116
  C:3F70H         LINE#         117
  C:3F70H         LINE#         118
  C:3F74H         LINE#         119
  C:3F74H         LINE#         120
  C:3F77H         LINE#         121
  C:3F84H         LINE#         122
  C:3F84H         LINE#         123
  C:3F8BH         LINE#         124
  C:3F96H         LINE#         125
  C:3F96H         LINE#         126
  C:3F9AH         LINE#         127
  C:3F9CH         LINE#         128
  C:3F9CH         LINE#         129
  C:3FA0H         LINE#         130
  C:3FA0H         LINE#         131
  C:3FA3H         LINE#         132
  C:3FB0H         LINE#         133
  C:3FB0H         LINE#         134
  C:3FB7H         LINE#         135
  C:3FC2H         LINE#         136
  C:3FC2H         LINE#         137
  C:3FC6H         LINE#         138
  C:3FC8H         LINE#         139
  C:3FC8H         LINE#         140
  C:3FCCH         LINE#         141
  C:3FCCH         LINE#         142
  C:3FDCH         LINE#         143
  C:3FDCH         LINE#         144
  C:3FE3H         LINE#         145
  C:3FEEH         LINE#         146
  C:3FEEH         LINE#         147
  C:3FF2H         LINE#         148
  C:3FF4H         LINE#         149
  C:3FF4H         LINE#         150
  C:3FF8H         LINE#         151
  C:3FF8H         LINE#         152
  C:3FFBH         LINE#         153
  C:4008H         LINE#         154
BL51 BANKED LINKER/LOCATER V6.22                                                      12/09/2013  13:21:20  PAGE 12


  C:4008H         LINE#         155
  C:400FH         LINE#         156
  C:401AH         LINE#         157
  C:401AH         LINE#         158
  C:401EH         LINE#         159
  C:4020H         LINE#         160
  C:4020H         LINE#         161
  C:4024H         LINE#         162
  C:4024H         LINE#         163
  C:4034H         LINE#         164
  C:4034H         LINE#         165
  C:403BH         LINE#         166
  C:4046H         LINE#         167
  C:4046H         LINE#         168
  C:404AH         LINE#         169
  C:404CH         LINE#         170
  C:404CH         LINE#         171
  C:4050H         LINE#         172
  C:4050H         LINE#         173
  C:4060H         LINE#         174
  C:4060H         LINE#         175
  C:4067H         LINE#         176
  C:4072H         LINE#         177
  C:4072H         LINE#         178
  C:4076H         LINE#         179
  C:4078H         LINE#         180
  C:4078H         LINE#         181
  C:407CH         LINE#         182
  C:407CH         LINE#         183
  C:408CH         LINE#         184
  C:408CH         LINE#         185
  C:4093H         LINE#         186
  C:409EH         LINE#         187
  C:409EH         LINE#         188
  C:40A2H         LINE#         189
  C:40A4H         LINE#         190
  C:40A4H         LINE#         191
  C:40A8H         LINE#         192
  C:40A8H         LINE#         193
  C:40B8H         LINE#         194
  C:40B8H         LINE#         195
  C:40BFH         LINE#         196
  C:40CAH         LINE#         197
  C:40CAH         LINE#         198
  C:40CEH         LINE#         199
  C:40D0H         LINE#         200
  C:40D0H         LINE#         201
  C:40D4H         LINE#         202
  C:40D4H         LINE#         203
  C:40E4H         LINE#         204
  C:40E4H         LINE#         205
  C:40EBH         LINE#         206
  C:40F6H         LINE#         207
  C:40F6H         LINE#         208
  C:40FAH         LINE#         209
  C:40FCH         LINE#         210
  C:40FCH         LINE#         211
BL51 BANKED LINKER/LOCATER V6.22                                                      12/09/2013  13:21:20  PAGE 13


  C:4100H         LINE#         212
  C:4100H         LINE#         213
  C:4110H         LINE#         214
  C:4110H         LINE#         215
  C:4117H         LINE#         216
  C:4122H         LINE#         217
  C:4122H         LINE#         218
  C:4126H         LINE#         219
  C:4128H         LINE#         220
  C:4128H         LINE#         221
  C:412CH         LINE#         222
  C:412CH         LINE#         223
  C:413CH         LINE#         224
  C:413CH         LINE#         225
  C:4143H         LINE#         226
  C:414EH         LINE#         227
  C:414EH         LINE#         228
  C:4152H         LINE#         229
  C:4154H         LINE#         230
  C:4154H         LINE#         231
  C:4158H         LINE#         232
  C:4158H         LINE#         233
  C:4165H         LINE#         234
  C:4165H         LINE#         235
  C:416CH         LINE#         236
  C:4177H         LINE#         237
  C:4177H         LINE#         238
  C:417BH         LINE#         239
  C:417DH         LINE#         240
  C:417DH         LINE#         241
  C:4181H         LINE#         242
  C:4181H         LINE#         243
  C:418EH         LINE#         244
  C:418EH         LINE#         245
  C:4195H         LINE#         246
  C:41A0H         LINE#         247
  C:41A0H         LINE#         248
  C:41A4H         LINE#         249
  C:41A6H         LINE#         250
  C:41A6H         LINE#         251
  C:41BEH         LINE#         252
  C:41BEH         LINE#         253
  C:41BEH         LINE#         255
  -------         ENDPROC       DISPLAY_ID
  -------         PROC          LCD_INIT
  C:0003H         LINE#         260
  C:0003H         LINE#         261
  C:0003H         LINE#         262
  C:0013H         LINE#         263
  C:0013H         LINE#         264
  C:0019H         LINE#         265
  C:0021H         LINE#         266
  C:0029H         LINE#         267
  C:0031H         LINE#         268
  C:0039H         LINE#         269
  C:0040H         LINE#         270
  C:004BH         LINE#         271
BL51 BANKED LINKER/LOCATER V6.22                                                      12/09/2013  13:21:20  PAGE 14


  C:0055H         LINE#         273
  C:0060H         LINE#         274
  C:006BH         LINE#         275
  C:0076H         LINE#         276
  C:0081H         LINE#         277
  C:008CH         LINE#         278
  C:0097H         LINE#         279
  C:00A2H         LINE#         280
  C:00ADH         LINE#         281
  C:00B8H         LINE#         282
  C:00C3H         LINE#         284
  C:00CEH         LINE#         285
  C:00D9H         LINE#         286
  C:00E2H         LINE#         287
  C:00EDH         LINE#         289
  C:00F8H         LINE#         290
  C:0103H         LINE#         291
  C:010EH         LINE#         292
  C:0119H         LINE#         293
  C:0124H         LINE#         294
  C:012BH         LINE#         296
  C:0136H         LINE#         297
  C:0141H         LINE#         298
  C:014CH         LINE#         299
  C:0157H         LINE#         300
  C:0160H         LINE#         301
  C:016BH         LINE#         302
  C:0174H         LINE#         304
  C:017EH         LINE#         305
  C:0189H         LINE#         306
  C:0193H         LINE#         307
  C:019EH         LINE#         308
  C:01A7H         LINE#         309
  C:01B1H         LINE#         310
  C:01BCH         LINE#         311
  C:01C7H         LINE#         312
  C:01D1H         LINE#         313
  C:01D8H         LINE#         315
  C:01E3H         LINE#         316
  C:01EAH         LINE#         318
  C:01F3H         LINE#         319
  C:01FDH         LINE#         320
  C:0201H         LINE#         321
  C:0201H         LINE#         324
  C:0214H         LINE#         325
  C:0214H         LINE#         381
  C:0221H         LINE#         382
  C:022FH         LINE#         383
  C:023DH         LINE#         384
  C:024BH         LINE#         385
  C:0259H         LINE#         386
  C:0267H         LINE#         387
  C:0275H         LINE#         388
  C:027CH         LINE#         389
  C:028AH         LINE#         390
  C:0291H         LINE#         391
  C:029FH         LINE#         392
BL51 BANKED LINKER/LOCATER V6.22                                                      12/09/2013  13:21:20  PAGE 15


  C:02A6H         LINE#         393
  C:02B4H         LINE#         394
  C:02BBH         LINE#         395
  C:02C9H         LINE#         396
  C:02D0H         LINE#         397
  C:02DEH         LINE#         398
  C:02ECH         LINE#         399
  C:02FAH         LINE#         400
  C:0308H         LINE#         401
  C:0316H         LINE#         402
  C:0324H         LINE#         403
  C:0331H         LINE#         404
  C:033FH         LINE#         405
  C:034DH         LINE#         407
  C:035AH         LINE#         408
  C:0368H         LINE#         409
  C:0375H         LINE#         410
  C:0383H         LINE#         411
  C:0390H         LINE#         412
  C:039EH         LINE#         413
  C:03ABH         LINE#         415
  C:03B9H         LINE#         416
  C:03C7H         LINE#         417
  C:03D5H         LINE#         418
  C:03E3H         LINE#         419
  C:03F1H         LINE#         420
  C:03FFH         LINE#         421
  C:040DH         LINE#         422
  C:041AH         LINE#         423
  C:0428H         LINE#         424
  C:0436H         LINE#         426
  C:0444H         LINE#         428
  C:044BH         LINE#         429
  C:0459H         LINE#         430
  C:0460H         LINE#         431
  C:046EH         LINE#         432
  C:0475H         LINE#         433
  C:0483H         LINE#         434
  C:0483H         LINE#         436
  C:0486H         LINE#         437
  C:0493H         LINE#         438
  C:0493H         LINE#         440
  C:0493H         LINE#         441
  C:0493H         LINE#         442
  C:0493H         LINE#         443
  C:0493H         LINE#         444
  C:0493H         LINE#         445
  C:0493H         LINE#         446
  C:0493H         LINE#         447
  C:0493H         LINE#         448
  C:0493H         LINE#         449
  C:0493H         LINE#         450
  C:0493H         LINE#         451
  C:0493H         LINE#         452
  C:0493H         LINE#         453
  C:0493H         LINE#         454
  C:0493H         LINE#         455
BL51 BANKED LINKER/LOCATER V6.22                                                      12/09/2013  13:21:20  PAGE 16


  C:0493H         LINE#         456
  C:0493H         LINE#         457
  C:0493H         LINE#         458
  C:0493H         LINE#         459
  C:0493H         LINE#         460
  C:0493H         LINE#         461
  C:0493H         LINE#         462
  C:0493H         LINE#         465
  C:0493H         LINE#         466
  C:0493H         LINE#         467
  C:0493H         LINE#         468
  C:0493H         LINE#         469
  C:0493H         LINE#         470
  C:0493H         LINE#         471
  C:0493H         LINE#         472
  C:0493H         LINE#         473
  C:0493H         LINE#         474
  C:0493H         LINE#         475
  C:0493H         LINE#         478
  C:0493H         LINE#         479
  C:0493H         LINE#         480
  C:0493H         LINE#         481
  C:0493H         LINE#         482
  C:0493H         LINE#         483
  C:0493H         LINE#         484
  C:0493H         LINE#         485
  C:0493H         LINE#         486
  C:0493H         LINE#         487
  C:0493H         LINE#         488
  C:0493H         LINE#         490
  C:0495H         LINE#         491
  C:04A5H         LINE#         492
  C:04A5H         LINE#         494
  C:04AEH         LINE#         495
  C:04B9H         LINE#         496
  C:04C4H         LINE#         497
  C:04CFH         LINE#         498
  C:04DAH         LINE#         499
  C:04E5H         LINE#         500
  C:04F0H         LINE#         501
  C:04F9H         LINE#         502
  C:0502H         LINE#         503
  C:050BH         LINE#         504
  C:0516H         LINE#         505
  C:051FH         LINE#         506
  C:0528H         LINE#         507
  C:052FH         LINE#         508
  C:053AH         LINE#         509
  C:0541H         LINE#         510
  C:054CH         LINE#         511
  C:0553H         LINE#         512
  C:055EH         LINE#         513
  C:0565H         LINE#         514
  C:0570H         LINE#         515
  C:0577H         LINE#         516
  C:0582H         LINE#         519
  C:058BH         LINE#         520
BL51 BANKED LINKER/LOCATER V6.22                                                      12/09/2013  13:21:20  PAGE 17


  C:0596H         LINE#         521
  C:05A1H         LINE#         522
  C:05ACH         LINE#         523
  C:05B7H         LINE#         524
  C:05C0H         LINE#         525
  C:05CBH         LINE#         526
  C:05D6H         LINE#         527
  C:05E1H         LINE#         528
  C:05ECH         LINE#         529
  C:05F3H         LINE#         532
  C:05FCH         LINE#         533
  C:05FFH         LINE#         534
  C:0608H         LINE#         535
  C:0613H         LINE#         536
  C:061EH         LINE#         537
  C:0629H         LINE#         538
  C:0634H         LINE#         539
  C:063FH         LINE#         540
  C:064AH         LINE#         541
  C:064CH         LINE#         543
  C:064CH         LINE#         545
  C:065FH         LINE#         546
  C:065FH         LINE#         547
  C:0668H         LINE#         548
  C:0673H         LINE#         549
  C:067EH         LINE#         550
  C:0689H         LINE#         551
  C:0692H         LINE#         552
  C:069BH         LINE#         553
  C:06A4H         LINE#         554
  C:06ADH         LINE#         555
  C:06B8H         LINE#         556
  C:06C3H         LINE#         557
  C:06CCH         LINE#         558
  C:06D3H         LINE#         560
  C:06DEH         LINE#         561
  C:06E9H         LINE#         562
  C:06F0H         LINE#         564
  C:06FBH         LINE#         565
  C:0702H         LINE#         567
  C:070DH         LINE#         568
  C:0718H         LINE#         569
  C:0723H         LINE#         570
  C:072AH         LINE#         572
  C:0733H         LINE#         573
  C:073CH         LINE#         577
  C:0745H         LINE#         578
  C:0750H         LINE#         579
  C:075BH         LINE#         580
  C:0766H         LINE#         581
  C:0771H         LINE#         582
  C:077CH         LINE#         583
  C:0787H         LINE#         584
  C:0792H         LINE#         585
  C:079DH         LINE#         586
  C:07A8H         LINE#         590
  C:07B1H         LINE#         591
BL51 BANKED LINKER/LOCATER V6.22                                                      12/09/2013  13:21:20  PAGE 18


  C:07B4H         LINE#         592
  C:07BDH         LINE#         593
  C:07C8H         LINE#         595
  C:07CFH         LINE#         597
  C:07CFH         LINE#         598
  C:07CFH         LINE#         600
  C:07D2H         LINE#         601
  C:07E2H         LINE#         602
  C:07E2H         LINE#         603
  C:07EAH         LINE#         604
  C:07F5H         LINE#         605
  C:0800H         LINE#         610
  C:0809H         LINE#         611
  C:0814H         LINE#         612
  C:081DH         LINE#         613
  C:0826H         LINE#         614
  C:082FH         LINE#         615
  C:0838H         LINE#         616
  C:0841H         LINE#         617
  C:0848H         LINE#         619
  C:0853H         LINE#         620
  C:085EH         LINE#         621
  C:0869H         LINE#         622
  C:0874H         LINE#         623
  C:087FH         LINE#         624
  C:088AH         LINE#         625
  C:0895H         LINE#         626
  C:089EH         LINE#         627
  C:08A7H         LINE#         628
  C:08AAH         LINE#         629
  C:08B3H         LINE#         630
  C:08BEH         LINE#         631
  C:08C9H         LINE#         633
  C:08D4H         LINE#         634
  C:08DDH         LINE#         635
  C:08E6H         LINE#         636
  C:08EFH         LINE#         637
  C:08F8H         LINE#         638
  C:0901H         LINE#         639
  C:090AH         LINE#         640
  C:0913H         LINE#         641
  C:091EH         LINE#         642
  C:0927H         LINE#         643
  C:0932H         LINE#         644
  C:093DH         LINE#         645
  C:0948H         LINE#         646
  C:094AH         LINE#         647
  C:094AH         LINE#         649
  C:095DH         LINE#         650
  C:095DH         LINE#         651
  C:0963H         LINE#         652
  C:0969H         LINE#         653
  C:0970H         LINE#         654
  C:0977H         LINE#         655
  C:097EH         LINE#         656
  C:0985H         LINE#         657
  C:098CH         LINE#         658
BL51 BANKED LINKER/LOCATER V6.22                                                      12/09/2013  13:21:20  PAGE 19


  C:0993H         LINE#         659
  C:099AH         LINE#         660
  C:09A1H         LINE#         661
  C:09A8H         LINE#         662
  C:09AFH         LINE#         663
  C:09B6H         LINE#         664
  C:09BDH         LINE#         665
  C:09C4H         LINE#         666
  C:09CBH         LINE#         667
  C:09D1H         LINE#         668
  C:09D8H         LINE#         669
  C:09DFH         LINE#         670
  C:09E6H         LINE#         671
  C:09EDH         LINE#         672
  C:09F4H         LINE#         673
  C:09FAH         LINE#         674
  C:0A00H         LINE#         675
  C:0A07H         LINE#         676
  C:0A0EH         LINE#         677
  C:0A15H         LINE#         678
  C:0A1CH         LINE#         679
  C:0A23H         LINE#         680
  C:0A2AH         LINE#         681
  C:0A31H         LINE#         682
  C:0A38H         LINE#         683
  C:0A3FH         LINE#         684
  C:0A46H         LINE#         685
  C:0A4DH         LINE#         686
  C:0A54H         LINE#         687
  C:0A5BH         LINE#         688
  C:0A62H         LINE#         689
  C:0A68H         LINE#         690
  C:0A6FH         LINE#         691
  C:0A76H         LINE#         692
  C:0A7DH         LINE#         693
  C:0A84H         LINE#         694
  C:0A8BH         LINE#         695
  C:0A91H         LINE#         696
  C:0A98H         LINE#         697
  C:0A9FH         LINE#         698
  C:0AA6H         LINE#         699
  C:0AADH         LINE#         700
  C:0AB4H         LINE#         701
  C:0ABBH         LINE#         702
  C:0AC2H         LINE#         703
  C:0AC9H         LINE#         704
  C:0AD0H         LINE#         705
  C:0AD7H         LINE#         706
  C:0ADEH         LINE#         707
  C:0AE5H         LINE#         708
  C:0AECH         LINE#         709
  C:0AF3H         LINE#         710
  C:0AF9H         LINE#         711
  C:0AFFH         LINE#         712
  C:0B05H         LINE#         713
  C:0B0BH         LINE#         714
  C:0B12H         LINE#         715
BL51 BANKED LINKER/LOCATER V6.22                                                      12/09/2013  13:21:20  PAGE 20


  C:0B18H         LINE#         716
  C:0B1FH         LINE#         717
  C:0B26H         LINE#         718
  C:0B2DH         LINE#         719
  C:0B34H         LINE#         720
  C:0B3BH         LINE#         721
  C:0B42H         LINE#         722
  C:0B49H         LINE#         723
  C:0B50H         LINE#         724
  C:0B57H         LINE#         725
  C:0B5EH         LINE#         726
  C:0B65H         LINE#         727
  C:0B6CH         LINE#         728
  C:0B73H         LINE#         729
  C:0B7AH         LINE#         730
  C:0B81H         LINE#         731
  C:0B87H         LINE#         732
  C:0B8DH         LINE#         733
  C:0B94H         LINE#         734
  C:0B9BH         LINE#         735
  C:0BA2H         LINE#         736
  C:0BA8H         LINE#         737
  C:0BAEH         LINE#         738
  C:0BB4H         LINE#         739
  C:0BBBH         LINE#         740
  C:0BC2H         LINE#         741
  C:0BC9H         LINE#         742
  C:0BCDH         LINE#         743
  C:0BCDH         LINE#         745
  C:0BD0H         LINE#         746
  C:0BE0H         LINE#         747
  C:0BE0H         LINE#         748
  C:0BE6H         LINE#         749
  C:0BEFH         LINE#         750
  C:0BF8H         LINE#         751
  C:0C01H         LINE#         752
  C:0C08H         LINE#         755
  C:0C13H         LINE#         756
  C:0C1CH         LINE#         757
  C:0C27H         LINE#         758
  C:0C32H         LINE#         759
  C:0C3DH         LINE#         761
  C:0C48H         LINE#         762
  C:0C53H         LINE#         763
  C:0C5AH         LINE#         765
  C:0C65H         LINE#         766
  C:0C70H         LINE#         767
  C:0C77H         LINE#         770
  C:0C82H         LINE#         771
  C:0C8DH         LINE#         772
  C:0C98H         LINE#         773
  C:0CA3H         LINE#         774
  C:0CAEH         LINE#         775
  C:0CB9H         LINE#         776
  C:0CC4H         LINE#         777
  C:0CCFH         LINE#         778
  C:0CDAH         LINE#         779
BL51 BANKED LINKER/LOCATER V6.22                                                      12/09/2013  13:21:20  PAGE 21


  C:0CE5H         LINE#         780
  C:0CF0H         LINE#         781
  C:0CFBH         LINE#         782
  C:0D02H         LINE#         785
  C:0D0DH         LINE#         786
  C:0D18H         LINE#         787
  C:0D23H         LINE#         788
  C:0D2CH         LINE#         789
  C:0D37H         LINE#         790
  C:0D42H         LINE#         791
  C:0D4DH         LINE#         792
  C:0D56H         LINE#         793
  C:0D61H         LINE#         794
  C:0D6AH         LINE#         795
  C:0D75H         LINE#         796
  C:0D7EH         LINE#         797
  C:0D89H         LINE#         798
  C:0D94H         LINE#         799
  C:0D9FH         LINE#         800
  C:0DA8H         LINE#         801
  C:0DAFH         LINE#         804
  C:0DBAH         LINE#         805
  C:0DC5H         LINE#         806
  C:0DD0H         LINE#         807
  C:0DDBH         LINE#         809
  C:0DDFH         LINE#         811
  C:0DDFH         LINE#         813
  C:0DE2H         LINE#         814
  C:0DF2H         LINE#         815
  C:0DF2H         LINE#         817
  C:0DFBH         LINE#         818
  C:0E05H         LINE#         819
  C:0E0CH         LINE#         820
  C:0E17H         LINE#         821
  C:0E22H         LINE#         822
  C:0E2DH         LINE#         823
  C:0E36H         LINE#         824
  C:0E41H         LINE#         825
  C:0E4AH         LINE#         826
  C:0E53H         LINE#         827
  C:0E5CH         LINE#         828
  C:0E65H         LINE#         829
  C:0E6EH         LINE#         831
  C:0E77H         LINE#         832
  C:0E80H         LINE#         833
  C:0E89H         LINE#         834
  C:0E92H         LINE#         835
  C:0E99H         LINE#         836
  C:0EA4H         LINE#         837
  C:0EAFH         LINE#         838
  C:0EB6H         LINE#         839
  C:0EC1H         LINE#         840
  C:0EC8H         LINE#         841
  C:0ED3H         LINE#         842
  C:0EDEH         LINE#         843
  C:0EE5H         LINE#         844
  C:0EEEH         LINE#         845
BL51 BANKED LINKER/LOCATER V6.22                                                      12/09/2013  13:21:20  PAGE 22


  C:0EF7H         LINE#         847
  C:0F02H         LINE#         848
  C:0F0DH         LINE#         849
  C:0F18H         LINE#         852
  C:0F23H         LINE#         853
  C:0F2EH         LINE#         854
  C:0F39H         LINE#         855
  C:0F44H         LINE#         856
  C:0F4FH         LINE#         857
  C:0F5AH         LINE#         858
  C:0F65H         LINE#         860
  C:0F6EH         LINE#         861
  C:0F71H         LINE#         862
  C:0F7AH         LINE#         863
  C:0F85H         LINE#         864
  C:0F90H         LINE#         865
  C:0F9BH         LINE#         866
  C:0FA4H         LINE#         868
  C:0FAFH         LINE#         869
  C:0FB8H         LINE#         870
  C:0FC3H         LINE#         871
  C:0FCEH         LINE#         872
  C:0FD7H         LINE#         873
  C:0FE0H         LINE#         875
  C:0FEBH         LINE#         876
  C:0FF2H         LINE#         877
  C:0FFDH         LINE#         878
  C:1004H         LINE#         879
  C:100FH         LINE#         880
  C:1013H         LINE#         882
  C:1013H         LINE#         884
  C:1016H         LINE#         885
  C:1026H         LINE#         886
  C:1026H         LINE#         887
  C:1031H         LINE#         888
  C:103FH         LINE#         889
  C:104BH         LINE#         890
  C:1059H         LINE#         891
  C:1067H         LINE#         892
  C:1075H         LINE#         893
  C:1083H         LINE#         894
  C:1091H         LINE#         895
  C:109DH         LINE#         896
  C:10ABH         LINE#         897
  C:10B7H         LINE#         898
  C:10C3H         LINE#         899
  C:10D1H         LINE#         900
  C:10DFH         LINE#         901
  C:10EDH         LINE#         902
  C:10F9H         LINE#         903
  C:1105H         LINE#         904
  C:1111H         LINE#         905
  C:111DH         LINE#         906
  C:1129H         LINE#         907
  C:1137H         LINE#         908
  C:1143H         LINE#         909
  C:114FH         LINE#         910
BL51 BANKED LINKER/LOCATER V6.22                                                      12/09/2013  13:21:20  PAGE 23


  C:115DH         LINE#         911
  C:1169H         LINE#         912
  C:1177H         LINE#         913
  C:1185H         LINE#         914
  C:1193H         LINE#         915
  C:11A1H         LINE#         916
  C:11AFH         LINE#         917
  C:11BDH         LINE#         918
  C:11CBH         LINE#         919
  C:11D9H         LINE#         920
  C:11E7H         LINE#         921
  C:11F5H         LINE#         922
  C:1203H         LINE#         923
  C:120FH         LINE#         924
  C:121BH         LINE#         925
  C:122AH         LINE#         926
  C:122AH         LINE#         928
  C:123AH         LINE#         929
  C:123AH         LINE#         930
  C:123AH         LINE#         931
  C:123AH         LINE#         932
  C:123AH         LINE#         933
  C:123AH         LINE#         934
  C:123AH         LINE#         935
  C:123AH         LINE#         936
  C:123AH         LINE#         937
  C:123AH         LINE#         938
  C:123AH         LINE#         939
  C:123AH         LINE#         940
  C:123AH         LINE#         942
  C:123AH         LINE#         943
  C:123AH         LINE#         944
  C:123AH         LINE#         945
  C:123AH         LINE#         946
  C:123AH         LINE#         948
  C:123AH         LINE#         949
  C:123AH         LINE#         952
  C:123AH         LINE#         955
  C:123AH         LINE#         958
  C:123AH         LINE#         959
  C:123AH         LINE#         961
  C:123AH         LINE#         962
  C:123AH         LINE#         963
  C:123AH         LINE#         964
  C:123AH         LINE#         965
  C:123AH         LINE#         966
  C:123AH         LINE#         967
  C:123AH         LINE#         968
  C:123AH         LINE#         969
  C:123AH         LINE#         970
  C:123AH         LINE#         972
  C:123AH         LINE#         973
  C:123AH         LINE#         974
  C:123AH         LINE#         975
  C:123AH         LINE#         976
  C:123AH         LINE#         977
  C:123AH         LINE#         978
BL51 BANKED LINKER/LOCATER V6.22                                                      12/09/2013  13:21:20  PAGE 24


  C:123AH         LINE#         980
  C:123AH         LINE#         981
  C:123AH         LINE#         982
  C:123AH         LINE#         983
  C:123AH         LINE#         984
  C:123AH         LINE#         985
  C:123AH         LINE#         987
  C:123AH         LINE#         988
  C:123AH         LINE#         990
  C:123AH         LINE#         991
  C:123AH         LINE#         992
  C:123AH         LINE#         994
  C:124CH         LINE#         995
  C:124CH         LINE#         996
  C:1256H         LINE#         997
  C:1261H         LINE#         998
  C:126CH         LINE#         999
  C:1277H         LINE#         1000
  C:1280H         LINE#         1001
  C:128BH         LINE#         1002
  C:1294H         LINE#         1003
  C:129DH         LINE#         1004
  C:12A6H         LINE#         1005
  C:12AFH         LINE#         1006
  C:12B8H         LINE#         1008
  C:12C1H         LINE#         1009
  C:12CCH         LINE#         1010
  C:12D5H         LINE#         1011
  C:12DEH         LINE#         1012
  C:12E7H         LINE#         1014
  C:12F2H         LINE#         1015
  C:12FDH         LINE#         1018
  C:1308H         LINE#         1021
  C:1313H         LINE#         1024
  C:131EH         LINE#         1025
  C:1329H         LINE#         1027
  C:1334H         LINE#         1028
  C:133FH         LINE#         1029
  C:134AH         LINE#         1030
  C:1355H         LINE#         1031
  C:1360H         LINE#         1032
  C:136BH         LINE#         1033
  C:1376H         LINE#         1034
  C:1381H         LINE#         1035
  C:138CH         LINE#         1036
  C:1397H         LINE#         1038
  C:13A0H         LINE#         1039
  C:13A3H         LINE#         1040
  C:13ACH         LINE#         1041
  C:13B7H         LINE#         1042
  C:13C2H         LINE#         1043
  C:13CDH         LINE#         1044
  C:13D6H         LINE#         1046
  C:13DFH         LINE#         1047
  C:13E8H         LINE#         1048
  C:13F1H         LINE#         1049
  C:13FAH         LINE#         1050
BL51 BANKED LINKER/LOCATER V6.22                                                      12/09/2013  13:21:20  PAGE 25


  C:1403H         LINE#         1051
  C:140CH         LINE#         1053
  C:1417H         LINE#         1054
  C:1422H         LINE#         1056
  C:142AH         LINE#         1057
  C:142AH         LINE#         1058
  C:142AH         LINE#         1059
  C:142DH         LINE#         1060
  C:143DH         LINE#         1061
  C:143DH         LINE#         1062
  C:1447H         LINE#         1063
  C:1452H         LINE#         1066
  C:145DH         LINE#         1067
  C:1468H         LINE#         1068
  C:1473H         LINE#         1069
  C:147CH         LINE#         1070
  C:1487H         LINE#         1071
  C:1490H         LINE#         1072
  C:1499H         LINE#         1073
  C:14A4H         LINE#         1074
  C:14ADH         LINE#         1075
  C:14B6H         LINE#         1077
  C:14BFH         LINE#         1078
  C:14CAH         LINE#         1079
  C:14D3H         LINE#         1080
  C:14DCH         LINE#         1081
  C:14E7H         LINE#         1082
  C:14EEH         LINE#         1083
  C:14F9H         LINE#         1084
  C:1504H         LINE#         1085
  C:150BH         LINE#         1086
  C:1516H         LINE#         1087
  C:151DH         LINE#         1088
  C:1528H         LINE#         1089
  C:1533H         LINE#         1090
  C:153EH         LINE#         1091
  C:1545H         LINE#         1092
  C:154EH         LINE#         1093
  C:1557H         LINE#         1094
  C:155EH         LINE#         1096
  C:1567H         LINE#         1097
  C:1572H         LINE#         1098
  C:157DH         LINE#         1099
  C:1586H         LINE#         1100
  C:1591H         LINE#         1101
  C:159CH         LINE#         1102
  C:15A7H         LINE#         1103
  C:15B2H         LINE#         1104
  C:15BBH         LINE#         1105
  C:15C6H         LINE#         1106
  C:15CDH         LINE#         1107
  C:15D6H         LINE#         1108
  C:15D9H         LINE#         1109
  C:15E2H         LINE#         1110
  C:15EDH         LINE#         1112
  C:15F8H         LINE#         1113
  C:1603H         LINE#         1114
BL51 BANKED LINKER/LOCATER V6.22                                                      12/09/2013  13:21:20  PAGE 26


  C:160CH         LINE#         1115
  C:1615H         LINE#         1116
  C:161EH         LINE#         1117
  C:1627H         LINE#         1118
  C:1630H         LINE#         1119
  C:1639H         LINE#         1120
  C:1642H         LINE#         1122
  C:164DH         LINE#         1123
  C:1658H         LINE#         1125
  C:1658H         LINE#         1126
  C:1658H         LINE#         1128
  C:166BH         LINE#         1129
  C:166BH         LINE#         1130
  C:1675H         LINE#         1131
  C:1680H         LINE#         1132
  C:168BH         LINE#         1133
  C:1696H         LINE#         1135
  C:16A1H         LINE#         1136
  C:16AAH         LINE#         1137
  C:16B3H         LINE#         1138
  C:16BCH         LINE#         1139
  C:16C5H         LINE#         1140
  C:16CEH         LINE#         1142
  C:16D7H         LINE#         1143
  C:16E2H         LINE#         1144
  C:16EBH         LINE#         1145
  C:16F4H         LINE#         1146
  C:16FBH         LINE#         1147
  C:1706H         LINE#         1148
  C:1711H         LINE#         1149
  C:1718H         LINE#         1150
  C:1723H         LINE#         1151
  C:172AH         LINE#         1152
  C:1735H         LINE#         1153
  C:1740H         LINE#         1154
  C:174BH         LINE#         1155
  C:1752H         LINE#         1156
  C:175BH         LINE#         1157
  C:1766H         LINE#         1159
  C:176FH         LINE#         1160
  C:177AH         LINE#         1161
  C:1783H         LINE#         1162
  C:178EH         LINE#         1163
  C:1799H         LINE#         1164
  C:17A4H         LINE#         1165
  C:17AFH         LINE#         1166
  C:17BAH         LINE#         1167
  C:17C5H         LINE#         1168
  C:17D0H         LINE#         1170
  C:17D9H         LINE#         1171
  C:17DCH         LINE#         1172
  C:17E5H         LINE#         1173
  C:17F0H         LINE#         1174
  C:17FBH         LINE#         1175
  C:1806H         LINE#         1176
  C:180FH         LINE#         1178
  C:1818H         LINE#         1179
BL51 BANKED LINKER/LOCATER V6.22                                                      12/09/2013  13:21:20  PAGE 27


  C:1821H         LINE#         1180
  C:182AH         LINE#         1181
  C:1833H         LINE#         1182
  C:183CH         LINE#         1183
  C:1845H         LINE#         1185
  C:1850H         LINE#         1186
  C:185BH         LINE#         1187
  C:185BH         LINE#         1188
  C:185BH         LINE#         1190
  C:186EH         LINE#         1191
  C:186EH         LINE#         1193
  C:1876H         LINE#         1194
  C:187DH         LINE#         1195
  C:1888H         LINE#         1196
  C:1893H         LINE#         1197
  C:189EH         LINE#         1198
  C:18A9H         LINE#         1199
  C:18B4H         LINE#         1201
  C:18BFH         LINE#         1202
  C:18CAH         LINE#         1203
  C:18D5H         LINE#         1204
  C:18E0H         LINE#         1205
  C:18EBH         LINE#         1206
  C:18F6H         LINE#         1207
  C:1901H         LINE#         1208
  C:190CH         LINE#         1209
  C:1915H         LINE#         1210
  C:191EH         LINE#         1211
  C:1929H         LINE#         1212
  C:1932H         LINE#         1213
  C:193DH         LINE#         1214
  C:1946H         LINE#         1215
  C:194DH         LINE#         1216
  C:1958H         LINE#         1217
  C:1963H         LINE#         1218
  C:196AH         LINE#         1220
  C:1975H         LINE#         1221
  C:1980H         LINE#         1222
  C:198BH         LINE#         1223
  C:1996H         LINE#         1224
  C:199FH         LINE#         1225
  C:19AAH         LINE#         1226
  C:19B5H         LINE#         1228
  C:19BEH         LINE#         1229
  C:19C1H         LINE#         1230
  C:19CAH         LINE#         1231
  C:19D5H         LINE#         1233
  C:19E0H         LINE#         1234
  C:19EBH         LINE#         1235
  C:19F4H         LINE#         1236
  C:19FDH         LINE#         1238
  C:1A06H         LINE#         1239
  C:1A0FH         LINE#         1240
  C:1A18H         LINE#         1241
  C:1A21H         LINE#         1242
  C:1A2AH         LINE#         1244
  C:1A35H         LINE#         1245
BL51 BANKED LINKER/LOCATER V6.22                                                      12/09/2013  13:21:20  PAGE 28


  C:1A40H         LINE#         1246
  C:1A4BH         LINE#         1247
  C:1A54H         LINE#         1248
  C:1A5DH         LINE#         1249
  C:1A66H         LINE#         1251
  C:1A71H         LINE#         1252
  C:1A7CH         LINE#         1253
  C:1A87H         LINE#         1254
  C:1A90H         LINE#         1255
  C:1A99H         LINE#         1256
  C:1AA2H         LINE#         1257
  C:1AABH         LINE#         1258
  C:1AB4H         LINE#         1259
  C:1ABFH         LINE#         1260
  C:1AC6H         LINE#         1261
  C:1AD1H         LINE#         1262
  C:1AD8H         LINE#         1263
  C:1AE3H         LINE#         1264
  C:1AEAH         LINE#         1265
  C:1AEAH         LINE#         1267
  C:1AFDH         LINE#         1268
  C:1AFDH         LINE#         1269
  C:1B04H         LINE#         1270
  C:1B0CH         LINE#         1271
  C:1B14H         LINE#         1272
  C:1B1CH         LINE#         1274
  C:1B27H         LINE#         1275
  C:1B2EH         LINE#         1276
  C:1B39H         LINE#         1277
  C:1B44H         LINE#         1279
  C:1B4FH         LINE#         1280
  C:1B5AH         LINE#         1281
  C:1B65H         LINE#         1282
  C:1B70H         LINE#         1283
  C:1B7BH         LINE#         1284
  C:1B86H         LINE#         1285
  C:1B91H         LINE#         1286
  C:1B9CH         LINE#         1287
  C:1BA7H         LINE#         1288
  C:1BB2H         LINE#         1290
  C:1BBDH         LINE#         1291
  C:1BC6H         LINE#         1292
  C:1BD1H         LINE#         1293
  C:1BDAH         LINE#         1294
  C:1BE3H         LINE#         1295
  C:1BEAH         LINE#         1297
  C:1BF5H         LINE#         1298
  C:1C00H         LINE#         1299
  C:1C07H         LINE#         1301
  C:1C12H         LINE#         1302
  C:1C19H         LINE#         1304
  C:1C24H         LINE#         1305
  C:1C2FH         LINE#         1306
  C:1C3AH         LINE#         1307
  C:1C41H         LINE#         1309
  C:1C4CH         LINE#         1310
  C:1C57H         LINE#         1311
BL51 BANKED LINKER/LOCATER V6.22                                                      12/09/2013  13:21:20  PAGE 29


  C:1C62H         LINE#         1312
  C:1C6DH         LINE#         1313
  C:1C76H         LINE#         1314
  C:1C7FH         LINE#         1315
  C:1C88H         LINE#         1316
  C:1C93H         LINE#         1317
  C:1C9CH         LINE#         1318
  C:1C9FH         LINE#         1319
  C:1CA8H         LINE#         1320
  C:1CB3H         LINE#         1321
  C:1CBEH         LINE#         1322
  C:1CC9H         LINE#         1323
  C:1CD2H         LINE#         1326
  C:1CDDH         LINE#         1327
  C:1CE8H         LINE#         1328
  C:1CF3H         LINE#         1329
  C:1CFEH         LINE#         1330
  C:1D05H         LINE#         1332
  C:1D10H         LINE#         1333
  C:1D17H         LINE#         1334
  C:1D22H         LINE#         1335
  C:1D2DH         LINE#         1337
  C:1D36H         LINE#         1338
  C:1D3FH         LINE#         1339
  C:1D49H         LINE#         1340
  C:1D49H         LINE#         1342
  C:1D5CH         LINE#         1343
  C:1D5CH         LINE#         1344
  C:1D63H         LINE#         1345
  C:1D6BH         LINE#         1346
  C:1D72H         LINE#         1347
  C:1D7AH         LINE#         1348
  C:1D82H         LINE#         1349
  C:1D8AH         LINE#         1350
  C:1D92H         LINE#         1351
  C:1D9DH         LINE#         1352
  C:1DA4H         LINE#         1353
  C:1DAFH         LINE#         1354
  C:1DBAH         LINE#         1356
  C:1DC5H         LINE#         1357
  C:1DD0H         LINE#         1358
  C:1DDBH         LINE#         1359
  C:1DE6H         LINE#         1360
  C:1DF1H         LINE#         1361
  C:1DFCH         LINE#         1362
  C:1E07H         LINE#         1363
  C:1E12H         LINE#         1364
  C:1E1DH         LINE#         1365
  C:1E28H         LINE#         1369
  C:1E33H         LINE#         1370
  C:1E3EH         LINE#         1371
  C:1E49H         LINE#         1372
  C:1E54H         LINE#         1373
  C:1E5FH         LINE#         1374
  C:1E66H         LINE#         1375
  C:1E71H         LINE#         1376
  C:1E7CH         LINE#         1377
BL51 BANKED LINKER/LOCATER V6.22                                                      12/09/2013  13:21:20  PAGE 30


  C:1E87H         LINE#         1379
  C:1E92H         LINE#         1380
  C:1E9BH         LINE#         1382
  C:1EA6H         LINE#         1383
  C:1EAFH         LINE#         1384
  C:1EB8H         LINE#         1385
  C:1EC1H         LINE#         1386
  C:1ECCH         LINE#         1387
  C:1ED3H         LINE#         1388
  C:1EDEH         LINE#         1389
  C:1EE7H         LINE#         1390
  C:1EECH         LINE#         1391
  C:1EF5H         LINE#         1392
  C:1F00H         LINE#         1393
  C:1F09H         LINE#         1394
  C:1F12H         LINE#         1395
  C:1F1DH         LINE#         1397
  C:1F28H         LINE#         1398
  C:1F33H         LINE#         1399
  C:1F33H         LINE#         1401
  C:1F46H         LINE#         1402
  C:1F46H         LINE#         1403
  C:1F4EH         LINE#         1404
  C:1F55H         LINE#         1405
  C:1F60H         LINE#         1406
  C:1F6BH         LINE#         1407
  C:1F76H         LINE#         1408
  C:1F7DH         LINE#         1409
  C:1F88H         LINE#         1410
  C:1F93H         LINE#         1411
  C:1F9AH         LINE#         1412
  C:1FA5H         LINE#         1413
  C:1FACH         LINE#         1414
  C:1FB7H         LINE#         1415
  C:1FC2H         LINE#         1416
  C:1FC9H         LINE#         1417
  C:1FD4H         LINE#         1418
  C:1FDFH         LINE#         1419
  C:1FEAH         LINE#         1420
  C:1FF5H         LINE#         1421
  C:2000H         LINE#         1422
  C:2009H         LINE#         1423
  C:2014H         LINE#         1424
  C:201FH         LINE#         1425
  C:202AH         LINE#         1426
  C:2035H         LINE#         1427
  C:2040H         LINE#         1428
  C:204BH         LINE#         1429
  C:2056H         LINE#         1430
  C:2061H         LINE#         1431
  C:206CH         LINE#         1432
  C:2077H         LINE#         1433
  C:2082H         LINE#         1434
  C:208DH         LINE#         1435
  C:2098H         LINE#         1436
  C:20A3H         LINE#         1437
  C:20AEH         LINE#         1438
BL51 BANKED LINKER/LOCATER V6.22                                                      12/09/2013  13:21:20  PAGE 31


  C:20B9H         LINE#         1439
  C:20C4H         LINE#         1440
  C:20CFH         LINE#         1441
  C:20DAH         LINE#         1442
  C:20E5H         LINE#         1443
  C:20F0H         LINE#         1444
  C:20F9H         LINE#         1445
  C:20F9H         LINE#         1447
  C:210CH         LINE#         1448
  C:210CH         LINE#         1449
  C:2115H         LINE#         1450
  C:2120H         LINE#         1451
  C:212BH         LINE#         1452
  C:2136H         LINE#         1453
  C:2141H         LINE#         1454
  C:214CH         LINE#         1455
  C:2153H         LINE#         1456
  C:215EH         LINE#         1457
  C:2165H         LINE#         1458
  C:2170H         LINE#         1459
  C:217BH         LINE#         1460
  C:2182H         LINE#         1461
  C:218BH         LINE#         1462
  C:2196H         LINE#         1463
  C:21A1H         LINE#         1464
  C:21ACH         LINE#         1465
  C:21B7H         LINE#         1466
  C:21C2H         LINE#         1467
  C:21CDH         LINE#         1468
  C:21D8H         LINE#         1469
  C:21E3H         LINE#         1470
  C:21EEH         LINE#         1472
  C:21F9H         LINE#         1473
  C:2204H         LINE#         1474
  C:220FH         LINE#         1475
  C:2219H         LINE#         1476
  C:2224H         LINE#         1477
  C:222FH         LINE#         1478
  C:223AH         LINE#         1479
  C:2245H         LINE#         1480
  C:2250H         LINE#         1481
  C:225BH         LINE#         1482
  C:2266H         LINE#         1483
  C:2271H         LINE#         1484
  C:227CH         LINE#         1485
  C:2287H         LINE#         1486
  C:2292H         LINE#         1487
  C:229DH         LINE#         1488
  C:22A8H         LINE#         1489
  C:22A8H         LINE#         1491
  C:22B9H         LINE#         1492
  C:22B9H         LINE#         1493
  C:22BBH         LINE#         1494
  C:22C1H         LINE#         1495
  C:22C3H         LINE#         1496
  C:22CAH         LINE#         1497
  C:22CCH         LINE#         1498
BL51 BANKED LINKER/LOCATER V6.22                                                      12/09/2013  13:21:20  PAGE 32


  C:22CEH         LINE#         1499
  C:22D0H         LINE#         1500
  C:22D2H         LINE#         1501
  C:22D9H         LINE#         1504
  C:22E4H         LINE#         1505
  C:22EFH         LINE#         1506
  C:22F8H         LINE#         1507
  C:2303H         LINE#         1508
  C:230EH         LINE#         1509
  C:2319H         LINE#         1510
  C:2324H         LINE#         1511
  C:232FH         LINE#         1512
  C:233AH         LINE#         1513
  C:2345H         LINE#         1514
  C:2350H         LINE#         1515
  C:2357H         LINE#         1518
  C:2360H         LINE#         1519
  C:2369H         LINE#         1520
  C:2372H         LINE#         1521
  C:237DH         LINE#         1522
  C:2386H         LINE#         1523
  C:238FH         LINE#         1524
  C:239AH         LINE#         1525
  C:23A5H         LINE#         1528
  C:23B0H         LINE#         1529
  C:23BBH         LINE#         1530
  C:23C6H         LINE#         1531
  C:23D1H         LINE#         1532
  C:23DCH         LINE#         1534
  C:23E7H         LINE#         1535
  C:23F2H         LINE#         1536
  C:23FDH         LINE#         1537
  C:2408H         LINE#         1538
  C:2413H         LINE#         1539
  C:241EH         LINE#         1541
  C:2429H         LINE#         1542
  C:2432H         LINE#         1543
  C:243DH         LINE#         1544
  C:2446H         LINE#         1545
  C:244DH         LINE#         1546
  C:2458H         LINE#         1547
  C:2463H         LINE#         1548
  C:246EH         LINE#         1549
  C:2479H         LINE#         1550
  C:2484H         LINE#         1553
  C:248FH         LINE#         1554
  C:249AH         LINE#         1555
  C:24A1H         LINE#         1556
  C:24ACH         LINE#         1557
  C:24B7H         LINE#         1558
  C:24C0H         LINE#         1559
  C:24CBH         LINE#         1562
  C:24D6H         LINE#         1563
  C:24E1H         LINE#         1564
  C:24E8H         LINE#         1565
  C:24F3H         LINE#         1566
  C:24FAH         LINE#         1568
BL51 BANKED LINKER/LOCATER V6.22                                                      12/09/2013  13:21:20  PAGE 33


  C:2505H         LINE#         1569
  C:250CH         LINE#         1570
  C:2517H         LINE#         1571
  C:251EH         LINE#         1572
  C:2529H         LINE#         1573
  C:2530H         LINE#         1576
  C:253BH         LINE#         1577
  C:2546H         LINE#         1578
  C:254DH         LINE#         1579
  C:2558H         LINE#         1580
  C:2563H         LINE#         1581
  C:256AH         LINE#         1582
  C:2575H         LINE#         1585
  C:2580H         LINE#         1586
  C:258BH         LINE#         1587
  C:2594H         LINE#         1589
  C:259BH         LINE#         1590
  C:25A2H         LINE#         1592
  C:25B0H         LINE#         1593
  C:25B0H         LINE#         1594
  C:25B2H         LINE#         1595
  C:25B8H         LINE#         1596
  C:25BAH         LINE#         1597
  C:25C1H         LINE#         1598
  C:25C3H         LINE#         1599
  C:25C5H         LINE#         1600
  C:25C7H         LINE#         1601
  C:25C9H         LINE#         1602
  C:25D0H         LINE#         1605
  C:25DBH         LINE#         1606
  C:25E6H         LINE#         1607
  C:25EFH         LINE#         1608
  C:25FAH         LINE#         1609
  C:2605H         LINE#         1610
  C:2610H         LINE#         1611
  C:261BH         LINE#         1612
  C:2626H         LINE#         1613
  C:2631H         LINE#         1614
  C:263CH         LINE#         1615
  C:2647H         LINE#         1616
  C:264EH         LINE#         1619
  C:2657H         LINE#         1620
  C:2660H         LINE#         1621
  C:2669H         LINE#         1622
  C:2674H         LINE#         1623
  C:267DH         LINE#         1624
  C:2686H         LINE#         1625
  C:2691H         LINE#         1626
  C:269CH         LINE#         1629
  C:26A7H         LINE#         1630
  C:26B2H         LINE#         1631
  C:26BDH         LINE#         1632
  C:26C8H         LINE#         1633
  C:26D3H         LINE#         1635
  C:26DEH         LINE#         1636
  C:26E9H         LINE#         1637
  C:26F4H         LINE#         1638
BL51 BANKED LINKER/LOCATER V6.22                                                      12/09/2013  13:21:20  PAGE 34


  C:26FFH         LINE#         1639
  C:270AH         LINE#         1640
  C:2715H         LINE#         1642
  C:2720H         LINE#         1643
  C:2729H         LINE#         1644
  C:2734H         LINE#         1645
  C:273DH         LINE#         1646
  C:2744H         LINE#         1647
  C:274FH         LINE#         1648
  C:275AH         LINE#         1649
  C:2765H         LINE#         1650
  C:2770H         LINE#         1651
  C:277BH         LINE#         1654
  C:2786H         LINE#         1655
  C:2791H         LINE#         1656
  C:2798H         LINE#         1657
  C:27A3H         LINE#         1658
  C:27AEH         LINE#         1659
  C:27B7H         LINE#         1660
  C:27C2H         LINE#         1663
  C:27CDH         LINE#         1664
  C:27D8H         LINE#         1665
  C:27DFH         LINE#         1666
  C:27EAH         LINE#         1667
  C:27F1H         LINE#         1669
  C:27FCH         LINE#         1670
  C:2803H         LINE#         1671
  C:280EH         LINE#         1672
  C:2815H         LINE#         1673
  C:2820H         LINE#         1674
  C:2827H         LINE#         1677
  C:2832H         LINE#         1678
  C:283DH         LINE#         1679
  C:2844H         LINE#         1680
  C:284FH         LINE#         1681
  C:285AH         LINE#         1682
  C:2861H         LINE#         1683
  C:286CH         LINE#         1686
  C:2877H         LINE#         1687
  C:2882H         LINE#         1688
  C:288BH         LINE#         1690
  C:2892H         LINE#         1691
  C:2892H         LINE#         1693
  -------         ENDPROC       LCD_INIT
  -------         PROC          _LCD_ID
  X:002CH         SYMBOL        dat
  -------         DO            
  X:002EH         SYMBOL        temp
  X:0030H         SYMBOL        DH
  X:0032H         SYMBOL        DL
  X:002EH         SYMBOL        temp
  X:0030H         SYMBOL        DH
  X:0032H         SYMBOL        DL
  -------         ENDDO         
  -------         DO            
  X:002EH         SYMBOL        temp
  X:0030H         SYMBOL        DH
BL51 BANKED LINKER/LOCATER V6.22                                                      12/09/2013  13:21:20  PAGE 35


  X:0032H         SYMBOL        DL
  -------         ENDDO         
  C:57C2H         LINE#         1699
  C:57C9H         LINE#         1700
  C:57C9H         LINE#         1701
  C:57D4H         LINE#         1702
  C:57D4H         LINE#         1704
  C:57D9H         LINE#         1705
  C:57E3H         LINE#         1706
  C:57E9H         LINE#         1707
  C:57ECH         LINE#         1708
  C:57EFH         LINE#         1710
  C:57F1H         LINE#         1711
  C:57F3H         LINE#         1712
  C:57F5H         LINE#         1713
  C:57FBH         LINE#         1714
  C:5804H         LINE#         1716
  C:5806H         LINE#         1717
  C:5808H         LINE#         1718
  C:5810H         LINE#         1722
  C:5812H         LINE#         1723
  C:5814H         LINE#         1724
  C:5824H         LINE#         1726
  C:582BH         LINE#         1727
  C:582BH         LINE#         1728
  C:582BH         LINE#         1730
  C:582DH         LINE#         1731
  C:582DH         LINE#         1732
  C:582DH         LINE#         1734
  C:5837H         LINE#         1735
  C:583DH         LINE#         1736
  C:5840H         LINE#         1737
  C:5843H         LINE#         1739
  C:5845H         LINE#         1740
  C:5847H         LINE#         1741
  C:5849H         LINE#         1742
  C:584FH         LINE#         1744
  C:5858H         LINE#         1745
  C:5860H         LINE#         1748
  C:5862H         LINE#         1752
  C:5864H         LINE#         1754
  C:5874H         LINE#         1755
  C:587DH         LINE#         1756
  C:588DH         LINE#         1758
  C:588DH         LINE#         1759
  C:588DH         LINE#         1760
  -------         ENDPROC       _LCD_ID
  -------         PROC          _LCD_ID_61581
  X:002CH         SYMBOL        dat
  -------         DO            
  X:002EH         SYMBOL        temp
  D:0006H         SYMBOL        DH
  D:0004H         SYMBOL        DL
  -------         ENDDO         
  C:5541H         LINE#         1765
  C:5548H         LINE#         1766
  C:5548H         LINE#         1770
BL51 BANKED LINKER/LOCATER V6.22                                                      12/09/2013  13:21:20  PAGE 36


  C:554FH         LINE#         1771
  C:5555H         LINE#         1773
  C:555FH         LINE#         1774
  C:5565H         LINE#         1775
  C:5568H         LINE#         1776
  C:556BH         LINE#         1778
  C:556DH         LINE#         1779
  C:556FH         LINE#         1780
  C:5571H         LINE#         1781
  C:5577H         LINE#         1783
  C:557BH         LINE#         1784
  C:557FH         LINE#         1786
  C:5581H         LINE#         1787
  C:5584H         LINE#         1788
  C:5589H         LINE#         1790
  C:558BH         LINE#         1791
  C:558DH         LINE#         1792
  C:558FH         LINE#         1793
  C:5594H         LINE#         1795
  C:5598H         LINE#         1796
  C:559CH         LINE#         1798
  C:559EH         LINE#         1799
  C:55A1H         LINE#         1800
  C:55A6H         LINE#         1802
  C:55A8H         LINE#         1803
  C:55AAH         LINE#         1804
  C:55ACH         LINE#         1805
  C:55B1H         LINE#         1807
  C:55B5H         LINE#         1808
  C:55B9H         LINE#         1810
  C:55BBH         LINE#         1811
  C:55BEH         LINE#         1812
  C:55C3H         LINE#         1816
  C:55C5H         LINE#         1817
  C:55C7H         LINE#         1818
  C:55C9H         LINE#         1819
  C:55CEH         LINE#         1821
  C:55D2H         LINE#         1822
  C:55D6H         LINE#         1824
  C:55D8H         LINE#         1825
  C:55DBH         LINE#         1826
  C:55E0H         LINE#         1828
  C:55E8H         LINE#         1829
  C:55F1H         LINE#         1831
  C:55F3H         LINE#         1832
  C:55F5H         LINE#         1833
  C:55F7H         LINE#         1834
  C:55FCH         LINE#         1836
  C:5600H         LINE#         1837
  C:5604H         LINE#         1839
  C:5606H         LINE#         1840
  C:5609H         LINE#         1841
  C:560EH         LINE#         1845
  C:5610H         LINE#         1849
  C:561FH         LINE#         1851
  C:561FH         LINE#         1852
  -------         ENDPROC       _LCD_ID_61581
BL51 BANKED LINKER/LOCATER V6.22                                                      12/09/2013  13:21:20  PAGE 37


  -------         PROC          LCD_READ_ID61581
  -------         DO            
  D:0005H         SYMBOL        m
  D:0004H         SYMBOL        n
  -------         ENDDO         
  C:607DH         LINE#         1857
  C:607DH         LINE#         1858
  C:607DH         LINE#         1861
  C:607DH         LINE#         1862
  C:607DH         LINE#         1863
  C:6080H         LINE#         1864
  C:6087H         LINE#         1866
  C:6095H         LINE#         1869
  C:6095H         LINE#         1870
  C:6095H         LINE#         1871
  C:6095H         LINE#         1873
  C:6095H         LINE#         1874
  C:6095H         LINE#         1875
  C:6095H         LINE#         1877
  C:6098H         LINE#         1878
  -------         ENDPROC       LCD_READ_ID61581
  -------         PROC          _LCD_ID_9341
  D:0006H         SYMBOL        dat
  -------         DO            
  X:002CH         SYMBOL        temp
  X:002EH         SYMBOL        DH
  X:0030H         SYMBOL        DL
  -------         ENDDO         
  C:5A02H         LINE#         1885
  C:5A02H         LINE#         1886
  C:5A02H         LINE#         1887
  C:5A0DH         LINE#         1888
  C:5A0DH         LINE#         1889
  C:5A11H         LINE#         1890
  C:5A11H         LINE#         1891
  C:5A11H         LINE#         1893
  C:5A14H         LINE#         1894
  C:5A1AH         LINE#         1895
  C:5A1DH         LINE#         1896
  C:5A20H         LINE#         1898
  C:5A22H         LINE#         1899
  C:5A24H         LINE#         1900
  C:5A26H         LINE#         1901
  C:5A2CH         LINE#         1903
  C:5A2CH         LINE#         1904
  C:5A2CH         LINE#         1906
  C:5A2CH         LINE#         1907
  C:5A2CH         LINE#         1908
  C:5A2CH         LINE#         1910
  C:5A2CH         LINE#         1911
  C:5A2CH         LINE#         1912
  C:5A2CH         LINE#         1913
  C:5A2FH         LINE#         1915
  C:5A2FH         LINE#         1916
  C:5A2FH         LINE#         1918
  C:5A2FH         LINE#         1919
  C:5A2FH         LINE#         1920
BL51 BANKED LINKER/LOCATER V6.22                                                      12/09/2013  13:21:20  PAGE 38


  C:5A2FH         LINE#         1922
  C:5A2FH         LINE#         1923
  C:5A2FH         LINE#         1924
  C:5A2FH         LINE#         1925
  C:5A32H         LINE#         1927
  C:5A3BH         LINE#         1928
  C:5A43H         LINE#         1930
  C:5A45H         LINE#         1931
  C:5A4DH         LINE#         1932
  C:5A54H         LINE#         1934
  C:5A63H         LINE#         1935
  C:5A6CH         LINE#         1940
  C:5A6CH         LINE#         1941
  C:5A6CH         LINE#         1942
  C:5A6CH         LINE#         1943
  C:5A6FH         LINE#         1945
  C:5A78H         LINE#         1946
  C:5A80H         LINE#         1948
  C:5A82H         LINE#         1949
  C:5A8AH         LINE#         1950
  C:5A91H         LINE#         1954
  C:5A93H         LINE#         1957
  C:5AA8H         LINE#         1959
  C:5AA8H         LINE#         1960
  C:5AA8H         LINE#         1961
  -------         ENDPROC       _LCD_ID_9341
  -------         PROC          LCD_READ_8347ID
  -------         DO            
  D:0005H         SYMBOL        m
  D:0004H         SYMBOL        n
  -------         ENDDO         
  C:6003H         LINE#         1966
  C:6003H         LINE#         1967
  C:6003H         LINE#         1970
  C:6003H         LINE#         1971
  C:6006H         LINE#         1972
  C:600DH         LINE#         1973
  C:6017H         LINE#         1974
  C:601EH         LINE#         1975
  C:6025H         LINE#         1976
  C:6025H         LINE#         1978
  C:6025H         LINE#         1979
  C:6025H         LINE#         1980
  C:6025H         LINE#         1982
  C:6025H         LINE#         1983
  C:6025H         LINE#         1984
  C:6025H         LINE#         1986
  C:6028H         LINE#         1987
  -------         ENDPROC       LCD_READ_8347ID
  -------         PROC          LCD_READ_ID
  -------         DO            
  D:0005H         SYMBOL        m
  D:0004H         SYMBOL        n
  -------         ENDDO         
  C:602DH         LINE#         1993
  C:602DH         LINE#         1994
  C:602DH         LINE#         1997
BL51 BANKED LINKER/LOCATER V6.22                                                      12/09/2013  13:21:20  PAGE 39


  C:602DH         LINE#         1998
  C:6030H         LINE#         1999
  C:6037H         LINE#         2000
  C:6041H         LINE#         2001
  C:6048H         LINE#         2002
  C:604EH         LINE#         2003
  C:604EH         LINE#         2005
  C:604EH         LINE#         2006
  C:604EH         LINE#         2007
  C:604EH         LINE#         2009
  C:604EH         LINE#         2010
  C:604EH         LINE#         2011
  C:604EH         LINE#         2013
  C:6051H         LINE#         2014
  -------         ENDPROC       LCD_READ_ID
  -------         PROC          LCD_READ_ID9341
  -------         DO            
  D:0005H         SYMBOL        m
  D:0004H         SYMBOL        n
  -------         ENDDO         
  C:6056H         LINE#         2020
  C:6056H         LINE#         2021
  C:6056H         LINE#         2024
  C:6056H         LINE#         2025
  C:6056H         LINE#         2026
  C:6059H         LINE#         2027
  C:6060H         LINE#         2028
  C:6067H         LINE#         2029
  C:6075H         LINE#         2032
  C:6075H         LINE#         2033
  C:6075H         LINE#         2034
  C:6075H         LINE#         2036
  C:6075H         LINE#         2037
  C:6075H         LINE#         2038
  C:6075H         LINE#         2040
  C:6078H         LINE#         2041
  -------         ENDPROC       LCD_READ_ID9341
  C:60A0H         SYMBOL        L?0464
  -------         PROC          L?0463
  -------         ENDPROC       L?0463
  C:60A0H         SYMBOL        L?0464
  -------         PROC          HD_RESET
  C:60A6H         LINE#         2048
  C:60A6H         LINE#         2049
  C:60A6H         LINE#         2050
  C:60A8H         LINE#         2051
  C:60AFH         LINE#         2052
  C:60B1H         LINE#         2053
  -------         ENDPROC       HD_RESET
  C:5D11H         SYMBOL        L?0461
  -------         PROC          L?0460
  -------         ENDPROC       L?0460
  C:5D11H         SYMBOL        L?0461
  -------         PROC          _LCD_WRITE_CMD
  D:0007H         SYMBOL        cmd1
  D:0005H         SYMBOL        cmd2
  C:5D15H         LINE#         2059
BL51 BANKED LINKER/LOCATER V6.22                                                      12/09/2013  13:21:20  PAGE 40


  C:5D15H         LINE#         2060
  C:5D15H         LINE#         2061
  C:5D20H         LINE#         2062
  C:5D20H         LINE#         2063
  C:5D22H         LINE#         2064
  C:5D24H         LINE#         2065
  C:5D26H         LINE#         2066
  C:5D28H         LINE#         2067
  C:5D2AH         LINE#         2068
  C:5D2CH         LINE#         2070
  C:5D2EH         LINE#         2071
  C:5D30H         LINE#         2072
  C:5D30H         LINE#         2074
  C:5D30H         LINE#         2075
  C:5D30H         LINE#         2076
  C:5D32H         LINE#         2077
  C:5D32H         LINE#         2078
  C:5D34H         LINE#         2079
  C:5D36H         LINE#         2080
  C:5D38H         LINE#         2081
  C:5D3AH         LINE#         2082
  C:5D3CH         LINE#         2084
  C:5D40H         LINE#         2085
  C:5D42H         LINE#         2087
  C:5D44H         LINE#         2088
  C:5D46H         LINE#         2089
  C:5D46H         LINE#         2090
  -------         ENDPROC       _LCD_WRITE_CMD
  C:5D4AH         SYMBOL        L?0452
  C:5D64H         SYMBOL        L?0453
  -------         PROC          L?0451
  -------         ENDPROC       L?0451
  C:5D4AH         SYMBOL        L?0452
  C:5D64H         SYMBOL        L?0453
  -------         PROC          _LCD_WRITE_DATA
  D:0007H         SYMBOL        dataa
  D:0005H         SYMBOL        datab
  C:5D6CH         LINE#         2095
  C:5D6CH         LINE#         2096
  C:5D6CH         LINE#         2097
  C:5D77H         LINE#         2098
  C:5D77H         LINE#         2099
  C:5D79H         LINE#         2100
  C:5D7BH         LINE#         2101
  C:5D7DH         LINE#         2102
  C:5D7FH         LINE#         2103
  C:5D81H         LINE#         2104
  C:5D83H         LINE#         2106
  C:5D85H         LINE#         2107
  C:5D87H         LINE#         2108
  C:5D87H         LINE#         2110
  C:5D87H         LINE#         2111
  C:5D87H         LINE#         2112
  C:5D89H         LINE#         2113
  C:5D89H         LINE#         2114
  C:5D8BH         LINE#         2115
  C:5D8DH         LINE#         2116
BL51 BANKED LINKER/LOCATER V6.22                                                      12/09/2013  13:21:20  PAGE 41


  C:5D8FH         LINE#         2117
  C:5D91H         LINE#         2118
  C:5D93H         LINE#         2120
  C:5D97H         LINE#         2121
  C:5D99H         LINE#         2123
  C:5D9BH         LINE#         2124
  C:5D9DH         LINE#         2125
  C:5D9DH         LINE#         2126
  -------         ENDPROC       _LCD_WRITE_DATA
  -------         PROC          L?0462
  -------         ENDPROC       L?0462
  -------         PROC          _LLCD_WRITE_CMD
  D:0004H         SYMBOL        cmd
  C:5DB7H         LINE#         2131
  C:5DBBH         LINE#         2132
  C:5DBBH         LINE#         2133
  C:5DC6H         LINE#         2134
  C:5DC6H         LINE#         2135
  C:5DC8H         LINE#         2136
  C:5DCAH         LINE#         2137
  C:5DCCH         LINE#         2138
  C:5DCEH         LINE#         2139
  C:5DD2H         LINE#         2140
  C:5DD4H         LINE#         2142
  C:5DD6H         LINE#         2143
  C:5DD8H         LINE#         2144
  C:5DD8H         LINE#         2146
  C:5DD8H         LINE#         2147
  C:5DD8H         LINE#         2148
  C:5DDAH         LINE#         2149
  C:5DDAH         LINE#         2150
  C:5DDCH         LINE#         2151
  C:5DDEH         LINE#         2152
  C:5DE0H         LINE#         2153
  C:5DE2H         LINE#         2154
  C:5DE6H         LINE#         2156
  C:5DEAH         LINE#         2157
  C:5DECH         LINE#         2159
  C:5DEEH         LINE#         2160
  C:5DF0H         LINE#         2161
  C:5DF0H         LINE#         2162
  -------         ENDPROC       _LLCD_WRITE_CMD
  -------         PROC          L?0459
  -------         ENDPROC       L?0459
  -------         PROC          _LLCD_WRITE_DATA
  D:0004H         SYMBOL        dataa
  C:5BEAH         LINE#         2167
  C:5BEEH         LINE#         2168
  C:5BEEH         LINE#         2169
  C:5BF9H         LINE#         2170
  C:5BF9H         LINE#         2171
  C:5BFBH         LINE#         2172
  C:5BFDH         LINE#         2173
  C:5BFFH         LINE#         2174
  C:5C01H         LINE#         2175
  C:5C05H         LINE#         2176
  C:5C07H         LINE#         2178
BL51 BANKED LINKER/LOCATER V6.22                                                      12/09/2013  13:21:20  PAGE 42


  C:5C09H         LINE#         2179
  C:5C0BH         LINE#         2180
  C:5C0BH         LINE#         2182
  C:5C0BH         LINE#         2183
  C:5C0BH         LINE#         2184
  C:5C0DH         LINE#         2185
  C:5C0DH         LINE#         2186
  C:5C0FH         LINE#         2187
  C:5C11H         LINE#         2188
  C:5C13H         LINE#         2189
  C:5C15H         LINE#         2190
  C:5C19H         LINE#         2195
  C:5C1DH         LINE#         2196
  C:5C1FH         LINE#         2198
  C:5C21H         LINE#         2199
  C:5C23H         LINE#         2200
  C:5C23H         LINE#         2201
  -------         ENDPROC       _LLCD_WRITE_DATA
  C:5ED2H         SYMBOL        L?0445
  C:5F02H         SYMBOL        L?0446
  C:5F04H         SYMBOL        L?0447
  C:5F06H         SYMBOL        L?0448
  -------         PROC          L?0444
  -------         ENDPROC       L?0444
  C:5ED2H         SYMBOL        L?0445
  C:5F02H         SYMBOL        L?0446
  C:5F04H         SYMBOL        L?0447
  C:5F06H         SYMBOL        L?0448
  -------         PROC          _SENG_CMD_DAT
  D:0006H         SYMBOL        cmd
  D:0002H         SYMBOL        dataa
  C:5F0AH         LINE#         2207
  C:5F0EH         LINE#         2208
  C:5F0EH         LINE#         2209
  C:5F11H         LINE#         2210
  -------         ENDPROC       _SENG_CMD_DAT
  C:5B39H         SYMBOL        L?0450
  -------         PROC          L?0449
  -------         ENDPROC       L?0449
  C:5B39H         SYMBOL        L?0450
  -------         PROC          _GUI_SPRINTF_STRING
  X:002CH         SYMBOL        x
  X:002DH         SYMBOL        y
  X:002FH         SYMBOL        s
  X:0031H         SYMBOL        color
  X:0033H         SYMBOL        b_color
  C:5B4AH         LINE#         2216
  C:5B5AH         LINE#         2217
  C:5B5AH         LINE#         2218
  C:5B69H         LINE#         2219
  C:5B69H         LINE#         2220
  C:5B9AH         LINE#         2221
  C:5BA0H         LINE#         2222
  C:5BADH         LINE#         2225
  -------         ENDPROC       _GUI_SPRINTF_STRING
  -------         PROC          _GUI_SPRINTF_CHAR
  X:0035H         SYMBOL        x
BL51 BANKED LINKER/LOCATER V6.22                                                      12/09/2013  13:21:20  PAGE 43


  X:0036H         SYMBOL        y
  X:0038H         SYMBOL        c
  X:0039H         SYMBOL        color
  X:003BH         SYMBOL        b_color
  -------         DO            
  X:003DH         SYMBOL        s_x
  X:003EH         SYMBOL        s_y
  X:003FH         SYMBOL        temp
  D:0006H         SYMBOL        j
  -------         ENDDO         
  C:5287H         LINE#         2230
  C:5294H         LINE#         2231
  C:5294H         LINE#         2234
  C:5298H         LINE#         2235
  C:52A8H         LINE#         2236
  C:52A8H         LINE#         2237
  C:52C1H         LINE#         2238
  C:52C1H         LINE#         2239
  C:52C6H         LINE#         2240
  C:52D9H         LINE#         2241
  C:52E8H         LINE#         2243
  C:52F5H         LINE#         2244
  C:52F5H         LINE#         2245
  C:5309H         LINE#         2246
  C:5309H         LINE#         2247
  C:532EH         LINE#         2248
  C:532EH         LINE#         2249
  C:5340H         LINE#         2250
  C:5342H         LINE#         2252
  C:5342H         LINE#         2253
  C:5363H         LINE#         2254
  C:5363H         LINE#         2255
  C:5363H         LINE#         2256
  C:536AH         LINE#         2257
  C:536AH         LINE#         2258
  C:5372H         LINE#         2259
  -------         ENDPROC       _GUI_SPRINTF_CHAR
  -------         PROC          _GUI_POINT
  D:0007H         SYMBOL        x
  D:0004H         SYMBOL        y
  X:0040H         SYMBOL        color
  C:60D2H         LINE#         2264
  C:60D9H         LINE#         2265
  C:60D9H         LINE#         2266
  C:60DCH         LINE#         2267
  -------         ENDPROC       _GUI_POINT
  -------         PROC          _LCD_SETXY
  D:0006H         SYMBOL        x
  D:0082H         SYMBOL        y
  C:60E6H         LINE#         2273
  C:60ECH         LINE#         2274
  C:60ECH         LINE#         2275
  -------         ENDPROC       _LCD_SETXY
  -------         PROC          _LCD_SETWINDOW
  D:0001H         SYMBOL        x0
  X:0043H         SYMBOL        y0
  X:0045H         SYMBOL        x1
BL51 BANKED LINKER/LOCATER V6.22                                                      12/09/2013  13:21:20  PAGE 44


  X:0046H         SYMBOL        y1
  C:4BB3H         LINE#         2281
  C:4BBFH         LINE#         2282
  C:4BBFH         LINE#         2283
  C:4BCAH         LINE#         2284
  C:4BD3H         LINE#         2285
  C:4BE1H         LINE#         2286
  C:4BEFH         LINE#         2287
  C:4BFAH         LINE#         2288
  C:4BFAH         LINE#         2289
  C:4C05H         LINE#         2290
  C:4C0EH         LINE#         2291
  C:4C0EH         LINE#         2292
  C:4C21H         LINE#         2293
  C:4C21H         LINE#         2294
  C:4C21H         LINE#         2295
  C:4C21H         LINE#         2296
  C:4C21H         LINE#         2298
  C:4C21H         LINE#         2299
  C:4C21H         LINE#         2300
  C:4C21H         LINE#         2302
  C:4C21H         LINE#         2303
  C:4C2DH         LINE#         2304
  C:4C2DH         LINE#         2305
  C:4C33H         LINE#         2306
  C:4C38H         LINE#         2307
  C:4C3DH         LINE#         2309
  C:4C42H         LINE#         2310
  C:4C49H         LINE#         2311
  C:4C50H         LINE#         2313
  C:4C52H         LINE#         2314
  C:4C55H         LINE#         2315
  C:4C65H         LINE#         2316
  C:4C65H         LINE#         2317
  C:4C72H         LINE#         2318
  C:4C7CH         LINE#         2319
  C:4C8BH         LINE#         2320
  C:4C9CH         LINE#         2322
  C:4CA8H         LINE#         2323
  C:4CB7H         LINE#         2324
  C:4CBBH         LINE#         2325
  C:4CBEH         LINE#         2326
  C:4CC4H         LINE#         2327
  C:4CC4H         LINE#         2328
  C:4CCCH         LINE#         2329
  C:4CD7H         LINE#         2330
  C:4CE0H         LINE#         2331
  C:4CEDH         LINE#         2332
  C:4CFAH         LINE#         2333
  C:4D08H         LINE#         2334
  C:4D15H         LINE#         2335
  C:4D1EH         LINE#         2336
  C:4D1EH         LINE#         2337
  C:4D20H         LINE#         2339
  C:4D20H         LINE#         2340
  C:4D2BH         LINE#         2341
  C:4D39H         LINE#         2342
BL51 BANKED LINKER/LOCATER V6.22                                                      12/09/2013  13:21:20  PAGE 45


  C:4D40H         LINE#         2343
  C:4D40H         LINE#         2345
  -------         ENDPROC       _LCD_SETWINDOW
  -------         PROC          _LCD_TEST_SINGLECOLOR
  X:002CH         SYMBOL        colorH
  D:0001H         SYMBOL        colorL
  -------         DO            
  X:002DH         SYMBOL        i
  X:002FH         SYMBOL        j
  -------         ENDDO         
  C:4836H         LINE#         2350
  C:483CH         LINE#         2351
  C:483CH         LINE#         2353
  C:484CH         LINE#         2354
  C:484CH         LINE#         2355
  C:484EH         LINE#         2356
  C:484EH         LINE#         2357
  C:4851H         LINE#         2358
  C:4854H         LINE#         2360
  C:4854H         LINE#         2361
  C:4854H         LINE#         2362
  C:4854H         LINE#         2363
  C:4857H         LINE#         2366
  C:485CH         LINE#         2367
  C:485EH         LINE#         2368
  C:485EH         LINE#         2369
  C:486BH         LINE#         2370
  C:486BH         LINE#         2371
  C:486BH         LINE#         2372
  C:486BH         LINE#         2373
  C:486BH         LINE#         2374
  C:486BH         LINE#         2378
  C:486BH         LINE#         2379
  C:486BH         LINE#         2380
  C:486BH         LINE#         2381
  C:487DH         LINE#         2382
  C:487DH         LINE#         2383
  C:487DH         LINE#         2384
  C:487DH         LINE#         2385
  C:487DH         LINE#         2386
  C:4887H         LINE#         2390
  C:488CH         LINE#         2391
  C:4891H         LINE#         2392
  C:4893H         LINE#         2393
  C:48A0H         LINE#         2394
  C:48A0H         LINE#         2395
  C:48A9H         LINE#         2396
  C:48B4H         LINE#         2397
  C:48BEH         LINE#         2398
  C:48C9H         LINE#         2400
  C:48D2H         LINE#         2401
  C:48DCH         LINE#         2402
  C:48E0H         LINE#         2403
  C:48F0H         LINE#         2404
  C:48F0H         LINE#         2405
  C:48F0H         LINE#         2406
  C:48F0H         LINE#         2407
BL51 BANKED LINKER/LOCATER V6.22                                                      12/09/2013  13:21:20  PAGE 46


  C:48F0H         LINE#         2408
  C:48F0H         LINE#         2409
  C:48F0H         LINE#         2410
  C:48F3H         LINE#         2411
  C:48FCH         LINE#         2412
  C:4907H         LINE#         2413
  C:490BH         LINE#         2414
  C:491BH         LINE#         2415
  C:491BH         LINE#         2416
  C:491BH         LINE#         2417
  C:491BH         LINE#         2418
  C:491BH         LINE#         2419
  C:491BH         LINE#         2420
  C:491BH         LINE#         2421
  C:491EH         LINE#         2422
  C:4927H         LINE#         2423
  C:4932H         LINE#         2424
  C:4936H         LINE#         2425
  C:4945H         LINE#         2426
  C:4945H         LINE#         2427
  C:4945H         LINE#         2428
  C:4945H         LINE#         2429
  C:4945H         LINE#         2430
  C:4945H         LINE#         2432
  C:4945H         LINE#         2433
  C:4948H         LINE#         2434
  C:494DH         LINE#         2436
  C:494FH         LINE#         2439
  C:494FH         LINE#         2440
  C:494FH         LINE#         2441
  C:494FH         LINE#         2442
  C:4952H         LINE#         2443
  C:495CH         LINE#         2447
  C:4961H         LINE#         2448
  C:4966H         LINE#         2449
  C:496DH         LINE#         2450
  C:496DH         LINE#         2452
  C:497AH         LINE#         2453
  C:497AH         LINE#         2454
  C:497FH         LINE#         2455
  C:497FH         LINE#         2456
  C:4985H         LINE#         2457
  C:4985H         LINE#         2458
  C:498EH         LINE#         2459
  C:49A6H         LINE#         2460
  C:49BFH         LINE#         2461
  C:49BFH         LINE#         2462
  C:49BFH         LINE#         2463
  C:49C5H         LINE#         2464
  C:49C5H         LINE#         2465
  C:49CBH         LINE#         2466
  C:49CBH         LINE#         2467
  C:49D4H         LINE#         2468
  C:49ECH         LINE#         2470
  -------         ENDPROC       _LCD_TEST_SINGLECOLOR
  -------         PROC          _LLCD_TEST_SINGLECOLOR
  X:004FH         SYMBOL        color
BL51 BANKED LINKER/LOCATER V6.22                                                      12/09/2013  13:21:20  PAGE 47


  -------         DO            
  X:0051H         SYMBOL        i
  X:0053H         SYMBOL        j
  -------         ENDDO         
  C:4664H         LINE#         2486
  C:466BH         LINE#         2487
  C:466BH         LINE#         2489
  C:467BH         LINE#         2490
  C:467BH         LINE#         2491
  C:467DH         LINE#         2492
  C:467DH         LINE#         2493
  C:4680H         LINE#         2494
  C:4683H         LINE#         2496
  C:4683H         LINE#         2497
  C:4683H         LINE#         2498
  C:4683H         LINE#         2499
  C:4686H         LINE#         2502
  C:468BH         LINE#         2503
  C:468DH         LINE#         2504
  C:468DH         LINE#         2505
  C:469AH         LINE#         2506
  C:469AH         LINE#         2507
  C:469AH         LINE#         2508
  C:469AH         LINE#         2509
  C:469AH         LINE#         2510
  C:469AH         LINE#         2514
  C:469AH         LINE#         2515
  C:469AH         LINE#         2516
  C:469AH         LINE#         2517
  C:46ACH         LINE#         2518
  C:46ACH         LINE#         2519
  C:46ACH         LINE#         2520
  C:46ACH         LINE#         2521
  C:46ACH         LINE#         2522
  C:46B6H         LINE#         2526
  C:46BBH         LINE#         2527
  C:46C0H         LINE#         2528
  C:46C2H         LINE#         2529
  C:46CFH         LINE#         2530
  C:46CFH         LINE#         2531
  C:46D8H         LINE#         2532
  C:46E3H         LINE#         2533
  C:46EDH         LINE#         2534
  C:46F8H         LINE#         2536
  C:4701H         LINE#         2537
  C:470BH         LINE#         2538
  C:470FH         LINE#         2539
  C:471FH         LINE#         2540
  C:471FH         LINE#         2541
  C:471FH         LINE#         2542
  C:471FH         LINE#         2543
  C:471FH         LINE#         2544
  C:471FH         LINE#         2545
  C:471FH         LINE#         2546
  C:4722H         LINE#         2547
  C:472BH         LINE#         2548
  C:4736H         LINE#         2549
BL51 BANKED LINKER/LOCATER V6.22                                                      12/09/2013  13:21:20  PAGE 48


  C:473AH         LINE#         2550
  C:474AH         LINE#         2551
  C:474AH         LINE#         2552
  C:474AH         LINE#         2553
  C:474AH         LINE#         2554
  C:474AH         LINE#         2555
  C:474AH         LINE#         2556
  C:474AH         LINE#         2557
  C:474DH         LINE#         2558
  C:4756H         LINE#         2559
  C:4761H         LINE#         2560
  C:4765H         LINE#         2561
  C:4774H         LINE#         2562
  C:4774H         LINE#         2563
  C:4774H         LINE#         2564
  C:4774H         LINE#         2565
  C:4774H         LINE#         2566
  C:4774H         LINE#         2568
  C:4774H         LINE#         2569
  C:4777H         LINE#         2570
  C:477CH         LINE#         2572
  C:477EH         LINE#         2575
  C:477EH         LINE#         2576
  C:477EH         LINE#         2577
  C:477EH         LINE#         2578
  C:4781H         LINE#         2579
  C:478BH         LINE#         2583
  C:4790H         LINE#         2584
  C:4795H         LINE#         2585
  C:479CH         LINE#         2586
  C:479CH         LINE#         2588
  C:47A9H         LINE#         2589
  C:47A9H         LINE#         2590
  C:47AEH         LINE#         2591
  C:47AEH         LINE#         2592
  C:47B4H         LINE#         2593
  C:47B4H         LINE#         2594
  C:47BEH         LINE#         2595
  C:47D6H         LINE#         2596
  C:47EFH         LINE#         2597
  C:47EFH         LINE#         2598
  C:47EFH         LINE#         2599
  C:47F5H         LINE#         2600
  C:47F5H         LINE#         2601
  C:47FBH         LINE#         2602
  C:47FBH         LINE#         2603
  C:4805H         LINE#         2604
  C:481DH         LINE#         2606
  -------         ENDPROC       _LLCD_TEST_SINGLECOLOR
  -------         PROC          KEYPRESS
  C:6109H         LINE#         2622
  C:6109H         LINE#         2623
  C:6109H         LINE#         2624
  C:610CH         LINE#         2625
  C:6115H         LINE#         2626
  -------         ENDPROC       KEYPRESS
  C:5E13H         SYMBOL        L?0455
BL51 BANKED LINKER/LOCATER V6.22                                                      12/09/2013  13:21:20  PAGE 49


  C:5E19H         SYMBOL        L?0456
  -------         PROC          L?0454
  -------         ENDPROC       L?0454
  C:5E13H         SYMBOL        L?0455
  C:5E19H         SYMBOL        L?0456
  -------         PROC          _DELAYMS
  X:0055H         SYMBOL        value
  C:5E1DH         LINE#         2631
  C:5E24H         LINE#         2632
  C:5E24H         LINE#         2633
  C:5E2DH         LINE#         2634
  C:5E2DH         LINE#         2635
  C:5E34H         LINE#         2636
  C:5E3FH         LINE#         2637
  C:5E41H         LINE#         2638
  -------         ENDPROC       _DELAYMS
  -------         PROC          _DELAYUS
  D:0006H         SYMBOL        value1
  C:6116H         LINE#         2643
  C:6116H         LINE#         2644
  C:6116H         LINE#         2645
  C:611AH         LINE#         2646
  C:6121H         LINE#         2647
  -------         ENDPROC       _DELAYUS
  -------         ENDMOD        LCD_DRIVE

  -------         MODULE        TOUCH
  C:0000H         SYMBOL        _ICE_DUMMY_
  D:0090H         PUBLIC        P1
  D:00B0H         PUBLIC        P3
  X:0006H         PUBLIC        tp_dev
  C:41BFH         PUBLIC        _TP_Adj_Info_Show
  C:5626H         PUBLIC        _LCD_ShowNum
  C:60B8H         PUBLIC        _TP_Write_Byte
  C:5373H         PUBLIC        _TP_Scan
  D:00A8H         PUBLIC        IE
  C:5E8BH         PUBLIC        _TP_Read_XY
  C:445CH         PUBLIC        _LCD_SetPos
  D:00B8H         PUBLIC        IP
  X:0023H         PUBLIC        CMD_RDX
  X:0024H         PUBLIC        CMD_RDY
  B:00B0H.5       PUBLIC        TDIN
  D:0098H         PUBLIC        SCON
  C:5F95H         PUBLIC        Load_Drow_Dialog
  D:0088H         PUBLIC        TCON
  B:00B0H.4       PUBLIC        DOUT
  C:4D41H         PUBLIC        _Draw_Circle
  C:5045H         PUBLIC        _TP_Read_XY2
  C:4A05H         PUBLIC        _LCD_DrawLine
  X:0025H         PUBLIC        TP_REMIND_MSG_TBL
  C:5F69H         PUBLIC        _LCD_DrawPoint
  C:5898H         PUBLIC        _LCD_ShowString
  B:00B0H.6       PUBLIC        TCL
  B:00B0H.3       PUBLIC        PEN
  C:5161H         PUBLIC        _TP_Read_XOY
  D:00C8H         PUBLIC        T2CON
  C:5C24H         PUBLIC        _TP_Read_AD
BL51 BANKED LINKER/LOCATER V6.22                                                      12/09/2013  13:21:20  PAGE 50


  B:00B0H.7       PUBLIC        TCS
  C:5E42H         PUBLIC        _LCD_Pow
  X:0028H         PUBLIC        POINT_COLOR
  X:002AH         PUBLIC        BACK_COLOR
  C:2893H         PUBLIC        TP_Adjust
  C:5C88H         PUBLIC        _TP_Draw_Big_Point
  C:5467H         PUBLIC        _TP_Drow_Touch_Point
  D:00D0H         PUBLIC        PSW
  -------         PROC          _LCD_SETPOS
  X:006FH         SYMBOL        x0
  X:0071H         SYMBOL        x1
  X:0073H         SYMBOL        y0
  X:0075H         SYMBOL        y1
  C:445CH         LINE#         212
  C:446FH         LINE#         213
  C:446FH         LINE#         214
  C:447DH         LINE#         215
  C:448BH         LINE#         216
  C:4499H         LINE#         217
  C:44A7H         LINE#         219
  C:44B2H         LINE#         220
  C:44B2H         LINE#         221
  C:44C0H         LINE#         222
  C:44C9H         LINE#         223
  C:44C9H         LINE#         224
  C:44D7H         LINE#         225
  C:44D7H         LINE#         226
  C:44E4H         LINE#         227
  C:44F2H         LINE#         228
  C:44FFH         LINE#         229
  C:450DH         LINE#         230
  C:451AH         LINE#         231
  C:4528H         LINE#         232
  C:4535H         LINE#         233
  C:453EH         LINE#         234
  C:453EH         LINE#         235
  C:4540H         LINE#         236
  C:454BH         LINE#         237
  C:454BH         LINE#         238
  C:4558H         LINE#         239
  C:4566H         LINE#         240
  C:4573H         LINE#         241
  C:4581H         LINE#         242
  C:458EH         LINE#         243
  C:459CH         LINE#         244
  C:45A9H         LINE#         245
  C:45B7H         LINE#         246
  C:45B9H         LINE#         247
  C:45BCH         LINE#         248
  C:45C9H         LINE#         249
  C:45C9H         LINE#         250
  C:45CFH         LINE#         251
  C:45D8H         LINE#         252
  C:45E1H         LINE#         254
  C:45E8H         LINE#         255
  C:45F1H         LINE#         256
  C:45FAH         LINE#         258
BL51 BANKED LINKER/LOCATER V6.22                                                      12/09/2013  13:21:20  PAGE 51


  C:45FCH         LINE#         259
  C:45FEH         LINE#         260
  C:460BH         LINE#         261
  C:460BH         LINE#         262
  C:4611H         LINE#         263
  C:461AH         LINE#         264
  C:4623H         LINE#         266
  C:462AH         LINE#         267
  C:4633H         LINE#         268
  C:463CH         LINE#         270
  C:463EH         LINE#         271
  C:4640H         LINE#         273
  C:4640H         LINE#         274
  C:464EH         LINE#         275
  C:465CH         LINE#         276
  C:4663H         LINE#         277
  C:4663H         LINE#         279
  -------         ENDPROC       _LCD_SETPOS
  -------         PROC          _TP_WRITE_BYTE
  D:0007H         SYMBOL        num
  -------         DO            
  D:0006H         SYMBOL        count
  -------         ENDDO         
  C:60B8H         LINE#         307
  C:60B8H         LINE#         308
  C:60B8H         LINE#         310
  C:60BAH         LINE#         311
  C:60BAH         LINE#         312
  C:60BAH         LINE#         313
  C:60C2H         LINE#         314
  C:60C4H         LINE#         315
  C:60C8H         LINE#         316
  C:60CAH         LINE#         317
  C:60CCH         LINE#         318
  C:60D1H         LINE#         320
  -------         ENDPROC       _TP_WRITE_BYTE
  -------         PROC          _TP_READ_AD
  D:0007H         SYMBOL        CMD
  -------         DO            
  D:0005H         SYMBOL        count
  X:0053H         SYMBOL        Num
  -------         ENDDO         
  C:5C24H         LINE#         327
  C:5C24H         LINE#         328
  C:5C24H         LINE#         329
  C:5C26H         LINE#         330
  C:5C2BH         LINE#         331
  C:5C2DH         LINE#         332
  C:5C2FH         LINE#         333
  C:5C31H         LINE#         334
  C:5C34H         LINE#         335
  C:5C3BH         LINE#         336
  C:5C3DH         LINE#         337
  C:5C44H         LINE#         338
  C:5C46H         LINE#         339
  C:5C48H         LINE#         340
  C:5C4AH         LINE#         341
BL51 BANKED LINKER/LOCATER V6.22                                                      12/09/2013  13:21:20  PAGE 52


  C:5C4AH         LINE#         342
  C:5C57H         LINE#         343
  C:5C59H         LINE#         344
  C:5C5BH         LINE#         345
  C:5C68H         LINE#         346
  C:5C6DH         LINE#         347
  C:5C85H         LINE#         348
  C:5C87H         LINE#         349
  C:5C87H         LINE#         350
  -------         ENDPROC       _TP_READ_AD
  -------         PROC          _TP_READ_XOY
  X:0042H         SYMBOL        xy
  -------         DO            
  X:0043H         SYMBOL        i
  D:0006H         SYMBOL        j
  X:0045H         SYMBOL        buf
  X:004FH         SYMBOL        sum
  X:0051H         SYMBOL        temp
  -------         ENDDO         
  C:5161H         LINE#         360
  C:5165H         LINE#         361
  C:5165H         LINE#         364
  C:516BH         LINE#         366
  C:519BH         LINE#         367
  C:51B3H         LINE#         368
  C:51B3H         LINE#         369
  C:51C3H         LINE#         370
  C:51C3H         LINE#         371
  C:51E3H         LINE#         372
  C:51E3H         LINE#         373
  C:51F8H         LINE#         374
  C:520EH         LINE#         375
  C:5220H         LINE#         376
  C:5220H         LINE#         377
  C:5227H         LINE#         378
  C:5235H         LINE#         379
  C:523BH         LINE#         380
  C:5271H         LINE#         381
  C:5286H         LINE#         382
  C:5286H         LINE#         383
  -------         ENDPROC       _TP_READ_XOY
  -------         PROC          _TP_READ_XY
  X:003AH         SYMBOL        x
  X:003DH         SYMBOL        y
  -------         DO            
  X:0040H         SYMBOL        xtemp
  D:0006H         SYMBOL        ytemp
  -------         ENDDO         
  C:5E8BH         LINE#         388
  C:5E95H         LINE#         389
  C:5E95H         LINE#         391
  C:5EA3H         LINE#         392
  C:5EAAH         LINE#         394
  C:5EC0H         LINE#         395
  C:5ECFH         LINE#         396
  C:5ED1H         LINE#         397
  -------         ENDPROC       _TP_READ_XY
BL51 BANKED LINKER/LOCATER V6.22                                                      12/09/2013  13:21:20  PAGE 53


  -------         PROC          L?0145
  -------         ENDPROC       L?0145
  -------         PROC          _TP_READ_XY2
  X:002CH         SYMBOL        x
  X:002FH         SYMBOL        y
  -------         DO            
  X:0032H         SYMBOL        x1
  X:0034H         SYMBOL        y1
  X:0036H         SYMBOL        x2
  X:0038H         SYMBOL        y2
  D:0007H         SYMBOL        flag
  -------         ENDDO         
  C:5045H         LINE#         404
  C:504FH         LINE#         405
  C:504FH         LINE#         409
  C:5065H         LINE#         410
  C:506AH         LINE#         411
  C:5080H         LINE#         412
  C:5085H         LINE#         413
  C:5113H         LINE#         415
  C:5113H         LINE#         416
  C:5137H         LINE#         417
  C:515BH         LINE#         418
  C:515EH         LINE#         419
  C:5160H         LINE#         420
  -------         ENDPROC       _TP_READ_XY2
  -------         PROC          L?0143
  -------         ENDPROC       L?0143
  -------         PROC          _TP_DROW_TOUCH_POINT
  X:004FH         SYMBOL        x
  X:0051H         SYMBOL        y
  D:0002H         SYMBOL        color
  C:5467H         LINE#         427
  C:5474H         LINE#         428
  C:5474H         LINE#         429
  C:547DH         LINE#         430
  C:54A6H         LINE#         431
  C:54CBH         LINE#         432
  C:54E4H         LINE#         433
  C:54FDH         LINE#         434
  C:5516H         LINE#         435
  C:552FH         LINE#         436
  -------         ENDPROC       _TP_DROW_TOUCH_POINT
  -------         PROC          _TP_DRAW_BIG_POINT
  X:002CH         SYMBOL        x
  X:002EH         SYMBOL        y
  D:0002H         SYMBOL        color
  C:5C88H         LINE#         441
  C:5C95H         LINE#         442
  C:5C95H         LINE#         443
  C:5C9EH         LINE#         444
  C:5CA8H         LINE#         445
  C:5CBDH         LINE#         446
  C:5CD2H         LINE#         447
  -------         ENDPROC       _TP_DRAW_BIG_POINT
  -------         PROC          _TP_SCAN
  D:0007H         SYMBOL        tp
BL51 BANKED LINKER/LOCATER V6.22                                                      12/09/2013  13:21:20  PAGE 54


  C:5373H         LINE#         454
  C:5373H         LINE#         455
  C:5373H         LINE#         456
  C:5379H         LINE#         457
  C:5379H         LINE#         458
  C:5382H         LINE#         459
  C:538BH         LINE#         460
  C:538BH         LINE#         461
  C:53CFH         LINE#         462
  C:5412H         LINE#         463
  C:5412H         LINE#         464
  C:5418H         LINE#         465
  C:5418H         LINE#         466
  C:541BH         LINE#         467
  C:5428H         LINE#         468
  C:5435H         LINE#         469
  C:5435H         LINE#         470
  C:5437H         LINE#         471
  C:5437H         LINE#         472
  C:543DH         LINE#         473
  C:543DH         LINE#         474
  C:5440H         LINE#         475
  C:5442H         LINE#         476
  C:5442H         LINE#         477
  C:5448H         LINE#         478
  C:544CH         LINE#         479
  C:5452H         LINE#         480
  C:5456H         LINE#         481
  C:5456H         LINE#         482
  C:5456H         LINE#         483
  C:545CH         LINE#         484
  -------         ENDPROC       _TP_SCAN
  -------         PROC          _TP_ADJ_INFO_SHOW
  X:004FH         SYMBOL        x0
  X:0051H         SYMBOL        y0
  X:0053H         SYMBOL        x1
  X:0055H         SYMBOL        y1
  X:0057H         SYMBOL        x2
  X:0059H         SYMBOL        y2
  X:005BH         SYMBOL        x3
  X:005DH         SYMBOL        y3
  X:005FH         SYMBOL        fac
  C:41BFH         LINE#         489
  C:41D2H         LINE#         490
  C:41D2H         LINE#         491
  C:41DAH         LINE#         492
  C:41F7H         LINE#         493
  C:4215H         LINE#         494
  C:423DH         LINE#         495
  C:4265H         LINE#         496
  C:428DH         LINE#         497
  C:42B5H         LINE#         498
  C:42DDH         LINE#         499
  C:4305H         LINE#         500
  C:432DH         LINE#         501
  C:434AH         LINE#         502
  C:4367H         LINE#         503
BL51 BANKED LINKER/LOCATER V6.22                                                      12/09/2013  13:21:20  PAGE 55


  C:438AH         LINE#         504
  C:43ADH         LINE#         505
  C:43D0H         LINE#         506
  C:43F3H         LINE#         507
  C:4416H         LINE#         508
  C:4439H         LINE#         509
  -------         ENDPROC       _TP_ADJ_INFO_SHOW
  -------         PROC          TP_ADJUST
  -------         DO            
  X:002CH         SYMBOL        pos_temp
  X:003CH         SYMBOL        cnt
  D:0007H         SYMBOL        i
  X:003DH         SYMBOL        d1
  X:003FH         SYMBOL        d2
  X:0041H         SYMBOL        tem1
  X:0045H         SYMBOL        tem2
  X:0049H         SYMBOL        fac
  X:004DH         SYMBOL        outtime
  -------         ENDDO         
  C:2893H         LINE#         515
  C:2893H         LINE#         516
  C:2893H         LINE#         518
  C:2897H         LINE#         522
  C:289CH         LINE#         523
  C:289FH         LINE#         524
  C:28A6H         LINE#         525
  C:28ACH         LINE#         526
  C:28B1H         LINE#         527
  C:28B9H         LINE#         528
  C:28C0H         LINE#         529
  C:28C6H         LINE#         531
  C:28D2H         LINE#         532
  C:28D6H         LINE#         533
  C:28DEH         LINE#         535
  C:28DEH         LINE#         536
  C:28DEH         LINE#         537
  C:28EEH         LINE#         538
  C:28EEH         LINE#         539
  C:28FBH         LINE#         541
  C:28FBH         LINE#         542
  C:2900H         LINE#         543
  C:2906H         LINE#         545
  C:291DH         LINE#         546
  C:2931H         LINE#         547
  C:2936H         LINE#         549
  C:2948H         LINE#         550
  C:2948H         LINE#         551
  C:2948H         LINE#         552
  C:294DH         LINE#         553
  C:2955H         LINE#         554
  C:2957H         LINE#         555
  C:2957H         LINE#         556
  C:295CH         LINE#         557
  C:2966H         LINE#         558
  C:2968H         LINE#         559
  C:2968H         LINE#         560
  C:2977H         LINE#         561
BL51 BANKED LINKER/LOCATER V6.22                                                      12/09/2013  13:21:20  PAGE 56


  C:2986H         LINE#         562
  C:2989H         LINE#         563
  C:2989H         LINE#         565
  C:29A8H         LINE#         566
  C:29C7H         LINE#         567
  C:29E3H         LINE#         568
  C:29FFH         LINE#         569
  C:2A37H         LINE#         571
  C:2A56H         LINE#         572
  C:2A75H         LINE#         573
  C:2A91H         LINE#         574
  C:2AADH         LINE#         575
  C:2AE5H         LINE#         576
  C:2B1BH         LINE#         577
  C:2B65H         LINE#         578
  C:2B65H         LINE#         579
  C:2B65H         LINE#         580
  C:2B65H         LINE#         581
  C:2B65H         LINE#         582
  C:2B65H         LINE#         583
  C:2B68H         LINE#         584
  C:2B68H         LINE#         585
  C:2B87H         LINE#         586
  C:2BA6H         LINE#         587
  C:2BC2H         LINE#         588
  C:2BDEH         LINE#         589
  C:2C16H         LINE#         591
  C:2C35H         LINE#         592
  C:2C54H         LINE#         593
  C:2C70H         LINE#         594
  C:2C8CH         LINE#         595
  C:2CC4H         LINE#         596
  C:2CFAH         LINE#         597
  C:2D32H         LINE#         598
  C:2D32H         LINE#         599
  C:2D32H         LINE#         600
  C:2D32H         LINE#         601
  C:2D32H         LINE#         602
  C:2D32H         LINE#         603
  C:2D35H         LINE#         604
  C:2D35H         LINE#         607
  C:2D54H         LINE#         608
  C:2D73H         LINE#         609
  C:2D8FH         LINE#         610
  C:2DABH         LINE#         611
  C:2DE3H         LINE#         613
  C:2E02H         LINE#         614
  C:2E21H         LINE#         615
  C:2E3DH         LINE#         616
  C:2E59H         LINE#         617
  C:2E91H         LINE#         618
  C:2EC7H         LINE#         619
  C:2F02H         LINE#         620
  C:2F02H         LINE#         621
  C:2F06H         LINE#         622
  C:2F15H         LINE#         623
  C:2F24H         LINE#         624
BL51 BANKED LINKER/LOCATER V6.22                                                      12/09/2013  13:21:20  PAGE 57


  C:2F9FH         LINE#         625
  C:2FA2H         LINE#         626
  C:2FA2H         LINE#         628
  C:2FCEH         LINE#         629
  C:3018H         LINE#         631
  C:3044H         LINE#         632
  C:308EH         LINE#         633
  C:30CAH         LINE#         634
  C:30CAH         LINE#         635
  C:30CEH         LINE#         636
  C:30DDH         LINE#         637
  C:30ECH         LINE#         638
  C:3114H         LINE#         639
  C:3123H         LINE#         640
  C:3125H         LINE#         641
  C:3125H         LINE#         642
  C:3129H         LINE#         643
  C:312DH         LINE#         644
  C:3130H         LINE#         645
  C:3130H         LINE#         646
  C:3135H         LINE#         647
  C:3139H         LINE#         648
  C:3139H         LINE#         649
  C:313CH         LINE#         650
  C:313CH         LINE#         651
  C:3144H         LINE#         652
  C:314BH         LINE#         653
  C:3173H         LINE#         654
  C:317AH         LINE#         656
  C:3181H         LINE#         658
  C:3181H         LINE#         659
  C:3181H         LINE#         660
  C:3188H         LINE#         661
  C:3193H         LINE#         662
  C:31A1H         LINE#         663
  C:31A1H         LINE#         665
  -------         ENDPROC       TP_ADJUST
  -------         PROC          _LCD_DRAWLINE
  X:0053H         SYMBOL        x1
  D:0004H         SYMBOL        y1
  D:0002H         SYMBOL        x2
  X:0059H         SYMBOL        y2
  -------         DO            
  X:005BH         SYMBOL        t
  X:005DH         SYMBOL        xerr
  X:005FH         SYMBOL        yerr
  X:0061H         SYMBOL        delta_x
  X:0063H         SYMBOL        delta_y
  X:0065H         SYMBOL        distance
  X:0067H         SYMBOL        incx
  X:0069H         SYMBOL        incy
  X:006BH         SYMBOL        uRow
  X:006DH         SYMBOL        uCol
  -------         ENDDO         
  C:4A05H         LINE#         674
  C:4A0CH         LINE#         675
  C:4A0CH         LINE#         677
BL51 BANKED LINKER/LOCATER V6.22                                                      12/09/2013  13:21:20  PAGE 58


  C:4A16H         LINE#         679
  C:4A2AH         LINE#         680
  C:4A37H         LINE#         681
  C:4A44H         LINE#         682
  C:4A4AH         LINE#         683
  C:4A5EH         LINE#         684
  C:4A6FH         LINE#         685
  C:4A82H         LINE#         686
  C:4A9CH         LINE#         687
  C:4AA7H         LINE#         688
  C:4ABAH         LINE#         689
  C:4ADDH         LINE#         690
  C:4AE2H         LINE#         691
  C:4B00H         LINE#         692
  C:4B00H         LINE#         693
  C:4B10H         LINE#         694
  C:4B20H         LINE#         695
  C:4B30H         LINE#         696
  C:4B4AH         LINE#         697
  C:4B4AH         LINE#         698
  C:4B5AH         LINE#         699
  C:4B6AH         LINE#         700
  C:4B6AH         LINE#         701
  C:4B84H         LINE#         702
  C:4B84H         LINE#         703
  C:4B94H         LINE#         704
  C:4BA4H         LINE#         705
  C:4BA4H         LINE#         706
  C:4BB2H         LINE#         707
  -------         ENDPROC       _LCD_DRAWLINE
  -------         PROC          _DRAW_CIRCLE
  X:0053H         SYMBOL        x0
  X:0055H         SYMBOL        y0
  D:0003H         SYMBOL        r
  -------         DO            
  X:0057H         SYMBOL        a
  X:0059H         SYMBOL        b
  X:005BH         SYMBOL        di
  -------         ENDDO         
  C:4D41H         LINE#         711
  C:4D4EH         LINE#         712
  C:4D4EH         LINE#         715
  C:4D5DH         LINE#         716
  C:4D6EH         LINE#         717
  C:4D8BH         LINE#         718
  C:4D8BH         LINE#         719
  C:4D96H         LINE#         720
  C:4DAAH         LINE#         721
  C:4DCDH         LINE#         722
  C:4DF0H         LINE#         723
  C:4E14H         LINE#         724
  C:4E38H         LINE#         725
  C:4E4BH         LINE#         726
  C:4E61H         LINE#         727
  C:4E6CH         LINE#         729
  C:4E97H         LINE#         731
  C:4E97H         LINE#         732
BL51 BANKED LINKER/LOCATER V6.22                                                      12/09/2013  13:21:20  PAGE 59


  C:4EC1H         LINE#         733
  C:4ECBH         LINE#         734
  C:4ECBH         LINE#         735
  C:4ECEH         LINE#         736
  -------         ENDPROC       _DRAW_CIRCLE
  C:5F59H         SYMBOL        L?0141
  C:5F5AH         SYMBOL        L?0142
  -------         PROC          L?0140
  -------         ENDPROC       L?0140
  C:5F59H         SYMBOL        L?0141
  C:5F5AH         SYMBOL        L?0142
  -------         PROC          _LCD_DRAWPOINT
  D:0004H         SYMBOL        x
  D:0082H         SYMBOL        y
  C:5F69H         LINE#         740
  C:5F71H         LINE#         741
  C:5F71H         LINE#         742
  C:5F8BH         LINE#         743
  -------         ENDPROC       _LCD_DRAWPOINT
  -------         PROC          L?0139
  -------         ENDPROC       L?0139
  -------         PROC          _LCD_SHOWSTRING
  X:0061H         SYMBOL        x
  X:0063H         SYMBOL        y
  X:0065H         SYMBOL        width
  X:0067H         SYMBOL        height
  X:0069H         SYMBOL        size
  X:006AH         SYMBOL        p
  -------         DO            
  X:006DH         SYMBOL        x0
  -------         ENDDO         
  C:5898H         LINE#         755
  C:58ABH         LINE#         756
  C:58ABH         LINE#         757
  C:58B5H         LINE#         758
  C:58BEH         LINE#         759
  C:58CEH         LINE#         760
  C:58E7H         LINE#         761
  C:58E7H         LINE#         762
  C:5910H         LINE#         763
  C:5924H         LINE#         764
  C:593BH         LINE#         765
  C:594BH         LINE#         766
  C:5956H         LINE#         767
  C:5959H         LINE#         768
  -------         ENDPROC       _LCD_SHOWSTRING
  -------         PROC          L?0144
  -------         ENDPROC       L?0144
  -------         PROC          _LCD_SHOWNUM
  X:0061H         SYMBOL        x
  X:0063H         SYMBOL        y
  X:0065H         SYMBOL        num
  X:0069H         SYMBOL        len
  X:006AH         SYMBOL        size
  -------         DO            
  X:006BH         SYMBOL        t
  X:006CH         SYMBOL        temp
BL51 BANKED LINKER/LOCATER V6.22                                                      12/09/2013  13:21:20  PAGE 60


  X:006DH         SYMBOL        enshow
  -------         ENDDO         
  C:5626H         LINE#         837
  C:5633H         LINE#         838
  C:5633H         LINE#         840
  C:5637H         LINE#         841
  C:5649H         LINE#         842
  C:5649H         LINE#         843
  C:567AH         LINE#         844
  C:568BH         LINE#         845
  C:568BH         LINE#         846
  C:568FH         LINE#         847
  C:568FH         LINE#         848
  C:56B3H         LINE#         849
  C:56B5H         LINE#         850
  C:56BAH         LINE#         852
  C:56BAH         LINE#         853
  C:56EAH         LINE#         854
  C:56F2H         LINE#         855
  -------         ENDPROC       _LCD_SHOWNUM
  -------         PROC          _LCD_POW
  X:006EH         SYMBOL        m
  X:006FH         SYMBOL        n
  -------         DO            
  X:0070H         SYMBOL        result
  -------         ENDDO         
  C:5E42H         LINE#         858
  C:5E49H         LINE#         859
  C:5E49H         LINE#         860
  C:5E51H         LINE#         861
  C:5E7DH         LINE#         862
  C:5E8AH         LINE#         863
  -------         ENDPROC       _LCD_POW
  -------         PROC          LOAD_DROW_DIALOG
  C:5F95H         LINE#         865
  C:5F95H         LINE#         866
  C:5F95H         LINE#         867
  C:5F9CH         LINE#         868
  C:5FA4H         LINE#         869
  C:5FC7H         LINE#         870
  C:5FCFH         LINE#         871
  -------         ENDPROC       LOAD_DROW_DIALOG
  -------         ENDMOD        TOUCH

  -------         MODULE        ?C?FPADD
  C:386CH         PUBLIC        ?C?FPADD
  C:3868H         PUBLIC        ?C?FPSUB
  -------         ENDMOD        ?C?FPADD

  -------         MODULE        ?C?FPMUL
  C:395DH         PUBLIC        ?C?FPMUL
  -------         ENDMOD        ?C?FPMUL

  -------         MODULE        ?C?FPDIV
  C:3A66H         PUBLIC        ?C?FPDIV
  -------         ENDMOD        ?C?FPDIV

BL51 BANKED LINKER/LOCATER V6.22                                                      12/09/2013  13:21:20  PAGE 61


  -------         MODULE        ?C?FPCMP
  C:3B05H         PUBLIC        ?C?FPCMP
  C:3B03H         PUBLIC        ?C?FPCMP3
  -------         ENDMOD        ?C?FPCMP

  -------         MODULE        ?C?FCAST
  C:3B7AH         PUBLIC        ?C?FCASTC
  C:3B75H         PUBLIC        ?C?FCASTI
  C:3B70H         PUBLIC        ?C?FCASTL
  -------         ENDMOD        ?C?FCAST

  -------         MODULE        ?C?CASTF
  C:3BAEH         PUBLIC        ?C?CASTF
  -------         ENDMOD        ?C?CASTF

  -------         MODULE        SQRT
  C:595EH         PUBLIC        _SQRT
  -------         ENDMOD        SQRT

  -------         MODULE        ?C?CLDPTR
  C:3C2FH         PUBLIC        ?C?CLDPTR
  -------         ENDMOD        ?C?CLDPTR

  -------         MODULE        ?C?UIDIV
  C:3C48H         PUBLIC        ?C?UIDIV
  -------         ENDMOD        ?C?UIDIV

  -------         MODULE        ?C?ISTPTR
  C:3C9DH         PUBLIC        ?C?ISTPTR
  -------         ENDMOD        ?C?ISTPTR

  -------         MODULE        ?C?LMUL
  C:3CBCH         PUBLIC        ?C?LMUL
  -------         ENDMOD        ?C?LMUL

  -------         MODULE        ?C?ULDIV
  C:3D47H         PUBLIC        ?C?ULDIV
  -------         ENDMOD        ?C?ULDIV

  -------         MODULE        ?C?LNEG
  C:3DD9H         PUBLIC        ?C?LNEG
  -------         ENDMOD        ?C?LNEG

  -------         MODULE        ?C?LLDPDATA
  C:3DE7H         PUBLIC        ?C?LLDPDATA
  -------         ENDMOD        ?C?LLDPDATA

  -------         MODULE        ?C?LSTPDATA
  C:3DF3H         PUBLIC        ?C?LSTPDATA
  -------         ENDMOD        ?C?LSTPDATA

  -------         MODULE        ?C?LSTKPDATA
  C:3DFFH         PUBLIC        ?C?LSTKPDATA
  -------         ENDMOD        ?C?LSTKPDATA

  -------         MODULE        ?C?ICALL
  C:3E18H         PUBLIC        ?C?ICALL
BL51 BANKED LINKER/LOCATER V6.22                                                      12/09/2013  13:21:20  PAGE 62


  C:3E1CH         PUBLIC        ?C?ICALL2
  -------         ENDMOD        ?C?ICALL

  -------         MODULE        ABS
  C:6122H         PUBLIC        _ABS
  -------         ENDMOD        ABS

*** WARNING L1: UNRESOLVED EXTERNAL SYMBOL
    SYMBOL:  _LCD_SHOWCHAR
    MODULE:  ..\OBJ\Touch.obj (TOUCH)

*** WARNING L1: UNRESOLVED EXTERNAL SYMBOL
    SYMBOL:  ?_LCD_SHOWCHAR?BYTE
    MODULE:  ..\OBJ\Touch.obj (TOUCH)

*** WARNING L2: REFERENCE MADE TO UNRESOLVED EXTERNAL
    SYMBOL:  ?_LCD_SHOWCHAR?BYTE
    MODULE:  ..\OBJ\Touch.obj (TOUCH)
    ADDRESS: 5933H

*** WARNING L2: REFERENCE MADE TO UNRESOLVED EXTERNAL
    SYMBOL:  _LCD_SHOWCHAR
    MODULE:  ..\OBJ\Touch.obj (TOUCH)
    ADDRESS: 5939H

*** WARNING L2: REFERENCE MADE TO UNRESOLVED EXTERNAL
    SYMBOL:  ?_LCD_SHOWCHAR?BYTE
    MODULE:  ..\OBJ\Touch.obj (TOUCH)
    ADDRESS: 56ABH

*** WARNING L2: REFERENCE MADE TO UNRESOLVED EXTERNAL
    SYMBOL:  ?_LCD_SHOWCHAR?BYTE
    MODULE:  ..\OBJ\Touch.obj (TOUCH)
    ADDRESS: 56E1H

*** WARNING L2: REFERENCE MADE TO UNRESOLVED EXTERNAL
    SYMBOL:  _LCD_SHOWCHAR
    MODULE:  ..\OBJ\Touch.obj (TOUCH)
    ADDRESS: 56E8H

Program Size: data=9.0 xdata=119 code=24878
LINK/LOCATE RUN COMPLETE.  7 WARNING(S),  0 ERROR(S)
